:020000040000FA
:0600000096EF3AF0120039
:060008005BEF14F0120092
:06005A0004006C750000BB
:10006000290200000800000074750000FE01000075
:100070000200000076750000FE0300000200000090
:0C0080005A750000E300000012000000B0
:10011000D9CFE6FFE1CFD9FF030EE126DF6ADF503A
:10012000F90F69E2DF50220DF3CF00F0F4CF01F0B8
:10013000000E0026010E0122010E00C0DBFF020EA0
:1001400001C0DBFF010EDBCFE9FFE828DBCFEAFFD0
:10015000EF6A010EDBCFE9FFE828DBCFEAFF210ED3
:10016000E926000EEA22EF90010EDBCFE9FFE82836
:10017000DBCFEAFF210EE926000EEA22EF82010E14
:10018000DBCFE9FFE828DBCFEAFF210EE926000EEE
:10019000EA22EF84010EDBCFE9FFE828DBCFEAFF9C
:1001A000210EE926000EEA22EF98010EDBCFE9FFCF
:1001B000E828DBCFEAFF210EE926000EEA22EF96BF
:1001C000010EDBCFE9FFE828DBCFEAFF0F0EE926BF
:1001D000000EEA22EF68010EDBCFE9FFE828DBCF53
:1001E000EAFF1F0EE926000EEA22580EEE6E020EFE
:1001F000EF6EDF2A94D70101EE6B040EEF6FF06B08
:10020000F16BF26BF36BE15EE7CFD9FF1200D9CF50
:10021000E6FFE1CFD9FF030EE126DF6ADF50F90FD9
:1002200001E386D0DF50220DF3CF00F0F4CF01F0D0
:10023000000E0026010E0122010E00C0DBFF020E9F
:1002400001C0DBFF010EDBCFE9FFE828DBCFEAFFCF
:10025000EF506CE1010EDBCFE9FFE828DBCFEAFFCE
:10026000010EEF6EDBCFE9FFE828DBCFEAFF0B0ED4
:10027000E926000EEA22E9CF00F0EACF01F0FD0EF8
:10028000DBCF02F0E828DBCF03F000C0E9FF01C0BC
:10029000EAFF02C0EEFF03C0EDFF010EDBCFE9FF76
:1002A000E828DBCFEAFF0D0EE926000EEA22EE6A0F
:1002B000EF6A010EDBCFE9FFE828DBCFEAFFEE5261
:1002C000060EE926000EEA22EE6AEE6AEE6AEF6A90
:1002D000010EDBCFE9FFE828DBCFEAFF210EE9269C
:1002E000000EEA22EF80010EDBCFE9FFE828DBCF2A
:1002F000EAFF210EE926000EEA22EF96010EDBCF7F
:10030000E9FFE828DBCFEAFF0F0EE926000EEA221C
:10031000EF68010EDBCFE9FFE828DBCFEAFF210E13
:10032000E926000EEA22EF82DF5003D0DF2A76D7DB
:10033000FE0EF36E040EE15EE7CFD9FF1200D9CFB7
:10034000E6FFE1CFD9FFFE0EDB50220DF3CFE9FF30
:10035000F4CFEAFF000EE926010EEA22EF50040A6C
:1003600001E102D0000E01D0010EF36EE552E7CF9D
:10037000D9FF1200D9CFE6FFE1CFD9FF020EE12667
:10038000FE0EDB50220DF3CF00F0F4CF01F0000E93
:100390000026010E012200C0DFFF010E01C0DBFFBD
:1003A000000EDBCFE9FFE828DBCFEAFFEF50040ABD
:1003B0000FE0000EDBCF00F0E828DBCF01F000C03B
:1003C000E6FF01C0E6FF64EC0DF0E550E55087D094
:1003D000FE0EDB50E66EC9EC04F0E550E66AE66A14
:1003E000E668110EE66E000EDBCFE9FFE828DBCFF2
:1003F000EAFF180EE926000EEA22EECF00F0EECF5B
:1004000001F0EECF02F0EECF03F000C0E6FF01C036
:10041000E6FF02C0E6FF03C0E6FFDBCFE9FFE82806
:10042000DBCFEAFF140EE926000EEA22EECF04F03D
:10043000EECF05F0EECF06F0EECF07F004C0E6FFFA
:1004400005C0E6FF06C0E6FF07C0E6FFDBCFE9FF19
:10045000E828DBCFEAFF0D0EE926000EEA22EECFF8
:1004600008F0EECF09F008C0E6FF09C0E6FFDBCFD9
:10047000E9FFE828DBCFEAFF0B0EE926000EEA22AF
:10048000EECF0AF0EECF0BF00AC0E6FF0BC0E6FF9E
:10049000DBCFE9FFE828DBCFEAFFEE52E9CF0CF033
:1004A000EACF0DF00CC0E6FF0DC0E6FFFAEC07F056
:1004B000120EE15E000EDBCFE9FFE828DBCFEAFF9A
:1004C000140EE926000EEA22EE2AEE22EE22EF2298
:1004D000DBCFE9FFE828DBCFEAFF050EEF6E030E66
:1004E000E15EE7CFD9FF1200D9CFE6FFE1CFD9FF18
:1004F000020EE126FE0EDB50220DF3CF00F0F4CF0A
:1005000001F0000E0026010E012200C0DFFF010EE7
:1005100001C0DBFF000EDBCFE9FFE828DBCFEAFFFD
:100520000F0EE926000EEA22EF50FF0A01E10ED07D
:10053000000EDBCFE9FFE828DBCFEAFF210EE9263A
:10054000000EEA22EFB2010EE86602D0F36A14D17F
:10055000000EDBCFE9FFE828DBCFEAFF100EE9262B
:10056000000EEA22EECF00F0EECF01F000C0E6FF71
:1005700001C0E6FFDBCFE9FFE828DBCFEAFF0F0E83
:10058000E926000EEA22EF50E66E100EE66E000E2F
:10059000DBCFE9FFE828DBCFEAFF180EE926000EE3
:1005A000EA22EECF02F0EECF03F0EECF04F0EECF72
:1005B00005F002C0E6FF03C0E6FF04C0E6FF05C089
:1005C000E6FFDBCFE9FFE828DBCFEAFF140EE926E0
:1005D000000EEA22EECF06F0EECF07F0EECF08F0E5
:1005E000EECF09F006C0E6FF07C0E6FF08C0E6FF51
:1005F00009C0E6FFDBCFE9FFE828DBCFEAFF0D0EFD
:10060000E926000EEA22EECF0AF0EECF0BF00AC088
:10061000E6FF0BC0E6FFDBCFE9FFE828DBCFEAFF10
:100620000B0EE926000EEA22EECF0CF0EECF0DF015
:100630000CC0E6FF0DC0E6FFDBCFE9FFE828DBCF0B
:10064000EAFFEE52E9CF0EF0EACF0FF00EC0E6FF60
:100650000FC0E6FFFAEC07F0120EE15E000EDBCFF2
:10066000E9FFE828DBCFEAFF140EE926000EEA22B4
:10067000EECFF6F1EECFF7F1EECFF8F1EECFF9F1E4
:10068000DBCFE9FFE828DBCFEAFF100EE926000EFA
:10069000EA22EECFF4F1EECFF5F1DBCFE9FFE82867
:1006A000DBCFEAFF140EE926000EEA22E9CF00F0C4
:1006B000EACF01F0DBCFE9FFE828DBCFEAFF100E3D
:1006C000E926000EEA22EECF02F0EECF03F000C0E2
:1006D000E9FF01C0EAFF0250EE260350EE22000EB1
:1006E000EE22EE22DBCFE9FFE828DBCFEAFF140E93
:1006F000E926000EEA22EECFF6F1EECFF7F1EECFCB
:10070000F8F1EECFF9F1DBCFE9FFE828DBCFEAFF24
:10071000210EE926000EEA22EF92DBCFE9FFE8285E
:10072000DBCFEAFF210EE926000EEA22EF98DBCFAD
:10073000E9FFE828DBCFEAFF0F0EE926000EEA22E8
:10074000EF50E66EE9EC28F0E550000EDBCFE9FF54
:10075000E828DBCFEAFF0F0EE926000EEA22EF6859
:10076000DBCFE9FFE828DBCFEAFF210EE926000E08
:10077000EA22EF82010EF36E030EE15EE7CFD9FFAE
:100780001200D9CFE6FFE1CFD9FFFE0EDB50220DDC
:10079000F3CFE9FFF4CFEAFF000EE926010EEA22CB
:1007A0000F0EE926000EEA22EF50FF0A04E19BEC4F
:1007B00027F0F35011D0FE0EDB50220DF3CFE9FFEE
:1007C000F4CFEAFF000EE926010EEA22210EE92607
:1007D000000EEA22EFB2010EF36EE552E7CFD9FF29
:1007E0001200D9CFE6FFE1CFD9FF040EE126FE0EBD
:1007F000DB50220DF3CF00F0F4CF01F0000E002605
:10080000010E0122020E00C0DBFF030E01C0DBFF60
:10081000020EDBCFE9FFE828DBCFEAFF0F0EE92667
:10082000000EEA22EF50FF0A3AE1020EDBCFE9FFA9
:10083000E828DBCFEAFF0F0EE926000EEA22EF6A76
:10084000020EDBCFE9FFE828DBCFEAFF0F0EE92637
:10085000000EEA22EF50E66E4BEC29F0E550020E56
:10086000DBCFE9FFE828DBCFEAFF100EE926000E18
:10087000EA22EE6AEF6A280EE66EE66A020EDBCF27
:10088000E9FFE828DBCFEAFF0F0EE926000EEA2297
:10089000EF50E66E39EC29F0E550E550E550020ED8
:1008A000DBCFE9FFE828DBCFEAFF100EE926000ED8
:1008B000EA22EECF00F0EECF01F000C0DFFF010E24
:1008C00001C0DBFF000EDBCF00F0E828DBCF01F03A
:1008D000C40E005C000E015802E3F36A55D0020E0C
:1008E000DBCFE9FFE828DBCFEAFF210EE926000E87
:1008F000EA22EF88FD0EDB50E66E86EC28F0E5502C
:10090000020EDBCFE9FFE828DBCFEAFF100EE92675
:10091000000EEA22EECF00F0EECF01F000C0DFFFC4
:10092000010E01C0DBFFDE4ADF2ADD52020EDBCF03
:10093000E9FFE828DBCFEAFF100EE926000EEA22E5
:10094000E9CF00F0EACF01F0DBCF02F0E828DBCFFF
:1009500003F000C0E9FF01C0EAFF02C0EEFF03C0E0
:10096000EDFF000EDBCF00F0E828DBCF01F0C40E76
:10097000005C000E015806E3FE0EDB50E66E74ECE0
:1009800002F0E550010EF36E050EE15EE7CFD9FFF0
:100990001200D9CFE6FFE1CFD9FF020EE126FE0E0D
:1009A000DB50220DF3CF00F0F4CF01F0000E002653
:1009B000010E012200C0DFFF010E01C0DBFF000EAF
:1009C000DBCFE9FFE828DBCFEAFF210EE926000EA6
:1009D000EA22EFB6010EE86602D0F36A0FD05FECB0
:1009E00028F0000EDBCFE9FFE828DBCFEAFF210E7D
:1009F000E926000EEA22EF96010EF36E030EE15E89
:100A0000E7CFD9FF1200D9CFE6FFE1CFD9FF020E21
:100A1000E126FE0EDB50220DF3CF00F0F4CF01F003
:100A2000000E0026010E012200C0DFFF010E01C0F2
:100A3000DBFF000EDBCFE9FFE828DBCFEAFF210E6A
:100A4000E926000EEA22EFB6010EE85044E0000E5F
:100A5000DBCFE9FFE828DBCFEAFF210EE926000E15
:100A6000EA22EFB4010EE85012E0280EE66EE66AC4
:100A7000F8EC28F0E550E550000EDBCFE9FFE82860
:100A8000DBCFEAFF210EE926000EEA22EF94000EEA
:100A9000DBCFE9FFE828DBCFEAFF210EE926000ED5
:100AA000EA22EF88FA0EDBCF00F0E828DBCF01F076
:100AB00000C0E6FF01C0E6FFFC0EDBCF02F0E82835
:100AC000DBCF03F002C0E6FF03C0E6FF29EC28F00D
:100AD000040EE15E02D0F36AF46A030EE15EE7CF32
:100AE000D9FF1200D9CFE6FFE1CFD9FF020EE126F0
:100AF000FE0EDB50220DF3CF00F0F4CF01F0000E1C
:100B00000026010E012200C0DFFF010E01C0DBFF45
:100B1000000EDBCFE9FFE828DBCFEAFF210EE92654
:100B2000000EEA22EFB6010EE85062E0000EDBCFC5
:100B3000E9FFE828DBCFEAFF210EE926000EEA22D2
:100B4000EFB4010EE85012E0280EE66EE66AF8EC0B
:100B500028F0E550E550000EDBCFE9FFE828DBCFB9
:100B6000EAFF210EE926000EEA22EF94000EDBCF09
:100B7000E9FFE828DBCFEAFF120EE926000EEA22A1
:100B8000EE5010E1ED500EE15FEC28F0000EDBCFEF
:100B9000E9FFE828DBCFEAFF210EE926000EEA2272
:100BA000EF9626D0000EDBCFE9FFE828DBCFEAFF87
:100BB000120EE926000EEA22EE06ED5AFC0EDBCFFD
:100BC00000F0E828DBCF01F000C0E6FF01C0E6FF3F
:100BD000F4EC27F0E550E5CF01F0E7CF00F0F3505B
:100BE00000C0E9FF01C0EAFFEF6E010EF36E01D015
:100BF000F36A030EE15EE7CFD9FF1200D9CFE6FF1B
:100C0000E1CFD9FFFE0EDB50220DF3CFE9FFF4CF89
:100C1000EAFF000EE926010EEA22210EE926000E67
:100C2000EA22EFB6010EF36EE552E7CFD9FF1200CC
:100C30001200D9CFE6FFE1CFD9FF240EE126140E32
:100C4000E66EE66AD9CF00F0DACF01F000C0E6FF29
:100C500001C0E6FF29EC28F0040EE15ED9CF00F0D8
:100C6000DACF01F000C0E6FF01C0E6FFB9EC0BF0FF
:100C7000E550E550FD0EDBCFE9FFE828DBCFEAFFCA
:100C8000060EE926000EEA22EECF00F0EECF01F0CC
:100C9000EECF02F0EECF03F0140E00C0DBFF150E16
:100CA00001C0DBFF160E02C0DBFF170E03C0DBFF27
:100CB000180E00C2DBFF190E01C2DBFF1A0E02C2C2
:100CC000DBFF1B0E03C2DBFF1C0EDB6A060EE76EAA
:100CD0001D0EE7CFDBFFFB0EDBCF00F0E828DBCFFC
:100CE00001F01E0E00C0DBFF1F0E01C0DBFF1E0E59
:100CF000DBCF02F0E828DBCF03F002C0E6FF03C041
:100D0000E6FF8BEC30F0F4CF01F0F3CF00F0E550CC
:100D1000E5501E0E00C0DBFF1F0E01C0DBFF0C0EF6
:100D2000E66EE66AD9CF02F0DACF03F0140E02269F
:100D300002C0E6FF03C0E6FF71EC31F0F4CF01F032
:100D4000F3CF00F0040EE15E001E011E210E00C074
:100D5000DBFF220E01C0DBFF240EE66EE66AF8EC34
:100D600028F0E550E550210EDB50E66E86EC28F0C9
:100D7000E550220EDB50E66E86EC28F0E550140EAE
:100D8000E66EE66AF8EC28F0E550E550FB0EDBCFA6
:100D900002F0E828DBCF03F002C0E6FF03C0E6FF65
:100DA000E3EC09F0F4CF01F0F3CF00F0E550E550AB
:100DB000210E00C0DBFF220E01C0DBFF210EDBCFC6
:100DC00000F0E828DBCF01F0100EDBCF02F0E828BE
:100DD000DBCF03F00050025C02E10150035803E056
:100DE0005FEC28F000D10C0EDB50E842E842E8420C
:100DF000E8420F0B3F0BE846E846EC0F006E230E6F
:100E000000C0DBFFFB0EDBCF02F0E828DBCF03F0F6
:100E1000230EDB50025C006E0350016A0156140E73
:100E2000005E000E015AFB0E00C0DBFFFC0E01C08D
:100E3000DBFF0C0EDB50E842E842E842E8420F0BD1
:100E40003F0BE846E846006E016A140E0026000ECD
:100E5000012200C0E6FF01C0E6FFF8EC28F0E550F3
:100E6000E550FD0EDBCF01F0E828DBCF02F001C03A
:100E7000E6FF02C0E6FFD9CF03F0DACF04F003C0EB
:100E8000E6FF04C0E6FF56EC0AF0040EE15EF3CF85
:100E900000F0200E00C0DBFFDB50020F01E280D02B
:100EA0005FEC28F0200EDB50FF0A01E09CD0D9CF88
:100EB00000F0DACF01F0080E0026FB0EDBCF02F0C7
:100EC000E828DBCF03F000C0E9FF01C0EAFF0250D1
:100ED000EE260350EE22000EEE22EE220D0EDB5027
:100EE000E842010BE85004E10D0EDB50010BE85025
:100EF00009E0080ED926000EDE2ADE22DE22DD22DF
:100F00000A0ED95EE66AE66AE668040EE66EDBCF94
:100F100000F0050EDBCF01F0060EDBCF02F0070E6E
:100F2000DBCF03F000C0E6FF01C0E6FF02C0E6FF32
:100F300003C0E6FF080EDBCF04F0090EDBCF05F09F
:100F40000A0EDBCF06F00B0EDBCF07F004C0E6FF86
:100F500005C0E6FF06C0E6FF07C0E6FF000EDBCFD8
:100F600008F0E828DBCF09F008C0E6FF09C0E6FF7B
:100F7000020EDBCF0AF0E828DBCF0BF00AC0E6FF59
:100F80000BC0E6FFFD0EDBCF0CF0E828DBCF0DF049
:100F90000CC0E6FF0DC0E6FFFAEC07F0120E22D0FF
:100FA000FB0EDBCF00F0E828DBCF01F000C0E6FF4E
:100FB00001C0E6FFD9CF02F0DACF03F002C0E6FFAE
:100FC00003C0E6FFFD0EDBCF04F0E828DBCF05F021
:100FD00004C0E6FF05C0E6FF200EDB50E66E0BEC1A
:100FE0000EF0070EE15E010EF36E250EE15EE7CF17
:100FF000D9FF1200D9CFE6FFE1CFD9FF260EE126B7
:101000009BEC27F0F35001E1FBD7FB0EDBCF00F0A8
:10101000E828DBCF01F0020E00C0DBFF030E01C0A9
:10102000DBFFF90EDBCF00F0E828DBCF01F0040E88
:1010300000C0DBFF050E01C0DBFFF50EDBCF00F0CB
:10104000F60EDBCF01F0F70EDBCF02F0F80EDBCFB0
:1010500003F0060E00C0DBFF070E01C0DBFF080E29
:1010600002C0DBFF090E03C0DBFFF10EDBCF00F097
:10107000F20EDBCF01F0F30EDBCF02F0F40EDBCF8C
:1010800003F00A0E00C0DBFF0B0E01C0DBFF0C0EED
:1010900002C0DBFF0D0E03C0DBFF0F0EDB9CDB9EEF
:1010A0000E0EDB90DB92DB94DB96F00EDBCF00F0D4
:1010B0000F0E00C0DBFF53EC29F0F4CF01F0F3CFAB
:1010C00000F0100E00C0DBFF110E01C0DBFF100EA0
:1010D000DBCF00F0E828DBCF01F000502808000E3D
:1010E00001540BE2D9CFE9FFDACFEAFF100EE9266F
:1010F000D80EEE26FF0EED2205D0100ED926DE6AA0
:10110000DD6AD95E120ED926DE6ADD6AD95E140E5A
:10111000D926DE6ADD6AD95ED9CF00F0DACF01F0D8
:10112000020E002600C0E6FF01C0E6FFB9EC0BF09E
:10113000E550E550D9CFE9FFDACFEAFFED0EE92619
:10114000140EEE26000EED22F00EDB50E8A21FD0AA
:10115000D9CFE9FFDACFEAFFED0EE926040EEE263D
:10116000000EED22020EE76E160EE7CFDBFF040E37
:10117000E76E170EE7CFDBFF180EDB6AFA0EE76E9D
:10118000190EE7CFDBFF0E0EDB98DB8A03D00E0EC5
:10119000DB88DB9ADB8CDB9E1A0E00C2DBFF1B0EAA
:1011A00001C2DBFF1C0E02C2DBFF1D0E03C2DBFF10
:1011B000FD0EDBCFE9FFE828DBCFEAFF060EE926CC
:1011C000000EEA22EECF00F0EECF01F0EECF02F0FB
:1011D000EECF03F01E0E00C0DBFF1F0E01C0DBFFD1
:1011E000200E02C0DBFF210E03C0DBFF220EDB6AF4
:1011F000060EE76E230EE7CFDBFFED0EDBCF00F030
:10120000E828DBCF01F0240E00C0DBFF250E01C073
:10121000DBFF240EDBCF02F0E828DBCF03F002C0B7
:10122000E6FF03C0E6FF8BEC30F0F4CF01F0F3CF24
:1012300000F0E550E550240E00C0DBFF250E01C094
:10124000DBFF0C0EE66EE66AD9CF02F0DACF03F0D0
:101250001A0E022602C0E6FF03C0E6FF71EC31F071
:10126000F4CF01F0F3CF00F0040EE15E001E011E8A
:10127000120E00C0DBFF130E01C0DBFF120EDBCF2E
:1012800000F0E828DBCF01F000C0DFFF010E01C055
:10129000DBFFEF0EDB50FF0A02E1EF0EDB6A140EFC
:1012A000E66EE66AEF0EDB50E66E39EC29F0E550AB
:1012B000E550E550ED0EDBCF00F0E828DBCF01F084
:1012C00000C0E6FF01C0E6FF060EE66EFD0EDBCFB6
:1012D00002F0E828DBCF03F002C0E6FF03C0E6FF20
:1012E0003BEC25F0050EE15E140EE66EE66AD9CF02
:1012F00000F0DACF01F0020E002600C0E6FF01C0C8
:10130000E6FFBCEC28F0040EE15EF00EDB50E8A234
:1013100011D0040EE66EE66AD9CF00F0DACF01F004
:10132000160E002600C0E6FF01C0E6FFBCEC28F068
:10133000040EE15E140EE66EE66AEF0EDB50E66E1A
:1013400039EC29F0E550E550E550ED0EDBCF02F029
:10135000E828DBCF03F002C0E6FF03C0E6FFE3ECC2
:1013600009F0F4CF01F0F3CF00F0E550E55000C0F4
:10137000DFFF010E01C0DBFF240EE66EE66AEF0E12
:10138000DB50E66E39EC29F0E550E550E550010EF2
:10139000DB50E66E86EC28F0E550DF50E66E86EC1A
:1013A00028F0E550E66AE66AEF0EDB50E66E39ECAF
:1013B00029F0E550E550E550E0EC28F0270EE15E1D
:1013C000E7CFD9FF1200D9CFE6FFE1CFD9FF040E56
:1013D000E126010EDF6EDE52DE6ADD6ADD52FD0EB1
:1013E000DBCF00F0DB06FE0EDBCF01F001E2DB0617
:1013F000005001E1015042E0F4EC27F0F3CF00F09F
:10140000030E00C0DBFFDF5018E1030EDBCF02F05C
:10141000010EDB500224016E010E01C0DBFFDB5028
:10142000006E030EDB50005C1FE2020EDB2ADB5075
:10143000E8661AD0010EDB2A17D0030EDBCF02F0CC
:10144000020EDB500224016E020E01C0DBFFDB50F6
:10145000006E030EDB50005C07E2010EDB2ADB505E
:10146000E86602D0020EDB2ADF50E86602D0010EE9
:1014700001D0000E006E00C0DFFFB1D7020EDB50BE
:10148000E81C006E020E00C0DBFF010EDB50E81C02
:10149000006E010E00C0DBFFDBCFF3FFE828DBCFDF
:1014A000F4FF050EE15EE7CFD9FF1200D9CFE6FFCA
:1014B000E1CFD9FF040EE126FE0EE76E030EE7CF63
:1014C000DBFF020EDB6A020EDB50F90F01E3A0D056
:1014D000020EDB50220DF3CF00F0F4CF01F0000E2E
:1014E0000026010E012200C0DFFF010E01C0DBFF5C
:1014F000000EDBCFE9FFE828DBCFEAFFEF5001E188
:1015000084D0000EDBCFE9FFE828DBCFEAFF0B0E2B
:10151000E926000EEA22EECF00F0EECF01F0FD0E3C
:10152000DBCFE9FFE828DBCFEAFFEE52EE52EECF49
:1015300002F0EECF03F00050025C01E066D00150F3
:10154000035863E1000EDBCFE9FFE828DBCFEAFFB9
:10155000EF50010A06E1020EDBCF00F0030E00C0DF
:10156000DBFF000EDBCFE9FFE828DBCFEAFF0D0E43
:10157000E926000EEA22EECF00F0EECF01F0FD0EDC
:10158000DBCFE9FFE828DBCFEAFFEECF02F0EECFBA
:1015900003F00050025C02E10150035801E035D035
:1015A000000EDBCFE9FFE828DBCFEAFFEE52060EA4
:1015B000E926000EEA22EECF04F0EECF05F0EECFE2
:1015C00006F0EECF07F0FB0EDBCFE9FFE828DBCF1C
:1015D000EAFF060EE926000EEA22EECF08F0EECF73
:1015E00009F0EECF0AF0EECF0BF000010451085CD9
:1015F00008E10551095805E106510A5802E1075171
:101600000B5801E002D0020EA5D0020EDB2A5BD7F8
:10161000030EDB50220DF3CF00F0F4CF01F0000EEB
:101620000026010E012200C0DFFF010E01C0DBFF1A
:10163000030EDB50FE0A01E18FD0000EDBCFE9FF85
:10164000E828DBCFEAFFEF50010AD87401E184D02B
:101650000A0EE66EE66AFB0EDBCF00F0E828DBCF71
:1016600001F000C0E6FF01C0E6FF000EDBCFE9FF9E
:10167000E828DBCFEAFFEE52E9CF02F0EACF03F031
:1016800002C0E6FF03C0E6FF10EC38F0060EE15E94
:10169000000EDBCFE9FFE828DBCFEAFF0B0EE926DF
:1016A000000EEA22E9CF00F0EACF01F0FD0EDBCF19
:1016B000E9FFE828DBCFEAFFEE52EE52EECF02F070
:1016C000EECF03F000C0E9FF01C0EAFF02C0EEFF69
:1016D00003C0EDFF000EDBCFE9FFE828DBCFEAFF18
:1016E0000D0EE926000EEA22E9CF00F0EACF01F064
:1016F000FD0EDBCFE9FFE828DBCFEAFFEECF02F0FB
:10170000EECF03F000C0E9FF01C0EAFF02C0EEFF28
:1017100003C0EDFF000EDBCFE9FFE828DBCFEAFFD7
:10172000210EE926000EEA22EF96DBCFE9FFE8283A
:10173000DBCFEAFF0F0EE926000EEA22EF68DBCFCF
:10174000E9FFE828DBCFEAFF210EE926000EEA22B6
:10175000EF82030EDB5007D0030EDB50FE0A02E1DE
:10176000F36802D0FE0EF36E050EE15EE7CFD9FFFF
:101770001200D9CFE6FFE1CFD9FFFD0EDBCFE9FFA5
:10178000E828DBCFEAFFE9CF00F0EACF01F000C0A4
:10179000E6FF01C0E6FFFD0EDBCFE9FFE828DBCF67
:1017A000EAFFEECF04F0EECF05F004C0E6FF05C07F
:1017B000E6FF8BEC30F0F4CF03F0F3CF02F0E5500E
:1017C000E550E550E5CF01F0E7CF00F000C0E9FFBC
:1017D00001C0EAFF02C0EEFF03C0EDFFFD0EDBCF4C
:1017E000E9FFE828DBCFEAFFEE52EE52E9CF00F046
:1017F000EACF01F000C0E6FF01C0E6FFFD0EDBCF3F
:10180000E9FFE828DBCFEAFFEE52EE52EECF04F01C
:10181000EECF05F004C0E6FF05C0E6FF8BEC30F02C
:10182000F4CF03F0F3CF02F0E550E550E550E5CFFB
:1018300001F0E7CF00F000C0E9FF01C0EAFF02C0FD
:10184000EEFF03C0EDFFFD0EDBCFE9FFE828DBCFA5
:10185000EAFF040EE926000EEA22E9CF00F0EACF03
:1018600001F000C0E6FF01C0E6FFFD0EDBCFE9FF9F
:10187000E828DBCFEAFF040EE926000EEA22EECFCD
:1018800006F0EECF07F0EECF08F0EECF09F006C07D
:10189000E6FF07C0E6FF08C0E6FF09C0E6FFB6ECBA
:1018A00030F0EECF02F0EECF03F0EECF04F0EECF4B
:1018B00005F0040EE15EE550E5CF01F0E7CF00F062
:1018C00000C0E9FF01C0EAFF02C0EEFF03C0EEFF67
:1018D00004C0EEFF05C0EFFFFD0EDBCFE9FFE828F7
:1018E000DBCFEAFF080EE926000EEA22E9CF00F07E
:1018F000EACF01F000C0E6FF01C0E6FFFD0EDBCF3E
:10190000E9FFE828DBCFEAFF080EE926000EEA220D
:10191000EECF06F0EECF07F0EECF08F0EECF09F0F5
:1019200006C0E6FF07C0E6FF08C0E6FF09C0E6FF05
:10193000B6EC30F0EECF02F0EECF03F0EECF04F0D5
:10194000EECF05F0040EE15EE550E5CF01F0E7CF04
:1019500000F000C0E9FF01C0EAFF02C0EEFF03C0D3
:10196000EEFF04C0EEFF05C0EFFFFD0EDBCFE9FF89
:10197000E828DBCFEAFF0E0EE926000EEA22E9CFC7
:1019800000F0EACF01F000C0E6FF01C0E6FFFD0E67
:10199000DBCFE9FFE828DBCFEAFF0E0EE926000ED9
:1019A000EA22EECF04F0EECF05F004C0E6FF05C05A
:1019B000E6FF8BEC30F0F4CF03F0F3CF02F0E5500C
:1019C000E550E550E5CF01F0E7CF00F000C0E9FFBA
:1019D00001C0EAFF02C0EEFF03C0EDFFFD0EDBCF4A
:1019E000E9FFE828DBCFEAFF100EE926000EEA2225
:1019F000E9CF00F0EACF01F000C0E6FF01C0E6FF4A
:101A0000FD0EDBCFE9FFE828DBCFEAFF100EE92669
:101A1000000EEA22EECF04F0EECF05F004C0E6FFA0
:101A200005C0E6FF8BEC30F0F4CF03F0F3CF02F00B
:101A3000E550E550E550E5CF01F0E7CF00F000C0FC
:101A4000E9FF01C0EAFF02C0EEFF03C0EDFFFD0E9B
:101A5000DBCFE9FFE828DBCFEAFF120EE926000E14
:101A6000EA22E9CF00F0EACF01F000C0E6FF01C0B2
:101A7000E6FFFD0EDBCFE9FFE828DBCFEAFF120E21
:101A8000E926000EEA22EECF04F0EECF05F004C006
:101A9000E6FF05C0E6FF8BEC30F0F4CF03F0F3CFA8
:101AA00002F0E550E550E550E5CF01F0E7CF00F05A
:101AB00000C0E9FF01C0EAFF02C0EEFF03C0EDFF76
:101AC000E552E7CFD9FF1200D9CFE6FFE1CFD9FF2A
:101AD000FD0EDBCFE9FFE828DBCFEAFF0F0EE9269A
:101AE000000EEA22EF50FF0A25E0FD0EDBCFE9FFF2
:101AF000E828DBCFEAFF0F0EE926000EEA22EF50BE
:101B0000E66EE9EC28F0E550FD0EDBCFE9FFE828B2
:101B1000DBCFEAFF0F0EE926000EEA22EF68FD0E8A
:101B2000DBCFE9FFE828DBCFEAFF210EE926000E34
:101B3000EA22EF82FD0EDBCFE9FFE828DBCFEAFFE8
:101B4000EE52060EE926000EEA22EE6AEE6AEE6A10
:101B5000EF6AFD0EDBCFE9FFE828DBCFEAFF0D0ED1
:101B6000E926000EEA22EE6AEF6AFD0EDBCFE9FFFE
:101B7000E828DBCFEAFF210EE926000EEA22EFB6C5
:101B8000010EE85002E05FEC28F0FD0EDBCFE9FF2C
:101B9000E828DBCFEAFF210EE926000EEA22EF96C5
:101BA000FD0EDBCFE9FFE828DBCFEAFF1F0EE926B9
:101BB000000EEA22580EEE6E020EEF6EFD0EDBCF27
:101BC000E9FFE828DBCFEAFF210EE926000EEA2232
:101BD000EF98FD0EDBCFE9FFE828DBCFEAFF210E0F
:101BE000E926000EEA22EF50010BE85009E0FD0E55
:101BF000DBCFE9FFE828DBCFEAFF010EEF6E07D06D
:101C0000FD0EDBCFE9FFE828DBCFEAFFEF6AE55204
:101C1000E7CFD9FF1200D9CFE6FFE1CFD9FF130EEE
:101C2000E126120EDB6AFE0EDB50220DF3CF00F030
:101C3000F4CF01F0000E0026010E0122100E00C0AC
:101C4000DBFF110E01C0DBFF100EDBCFE9FFE82840
:101C5000DBCFEAFF180EE926000EEA22EECF00F0F5
:101C6000EECF01F0EECF02F0EECF03F0080E00C091
:101C7000DBFF090E01C0DBFF0A0E02C0DBFF0B0E0B
:101C800003C0DBFF100EDBCFE9FFE828DBCFEAFF64
:101C9000140EE926000EEA22EECF00F0EECF01F09E
:101CA000EECF02F0EECF03F00C0E00C0DBFF0D0E06
:101CB00001C0DBFF0E0E02C0DBFF0F0E03C0DBFF17
:101CC000FA0EDBCFE9FFE828DBCFEAFF040EE926B6
:101CD000000EEA22EECF00F0EECF01F0EECF02F0E0
:101CE000EECF03F000C0DEFF01C0DDFF020E02C038
:101CF000DBFF030E03C0DBFFD9CF00F0DACF01F02A
:101D0000F80EDBCF02F0E828DBCF03F000C0E9FFDC
:101D100001C0EAFF0250EE260350EE22000EEE2232
:101D2000EE22100EDBCFE9FFE828DBCFEAFF140E2E
:101D3000E926000EEA22EECF00F0EECF01F0EECF62
:101D400002F0EECF03F0040E00C0DBFF050E01C071
:101D5000DBFF060E02C0DBFF070E03C0DBFFFA0E3F
:101D6000DBCFE9FFE828DBCFEAFF080EE926000E0B
:101D7000EA22EECFFAF1EECFFBF1EECFFCF1EECF9F
:101D8000FDF1100EDBCFE9FFE828DBCFEAFF1C0EE8
:101D9000E926000EEA22EF6A100EDBCFE9FFE82801
:101DA000DBCFEAFF1D0EE926000EEA22E9CF00F0A4
:101DB000EACF01F000C0E6FF01C0E6FF74EC3AF0A4
:101DC000F4CF03F0F3CF02F0E550E5CF01F0E7CF19
:101DD00000F000C0E9FF01C0EAFF02C0EEFF03C04F
:101DE000EDFF100EDBCFE9FFE828DBCFEAFF1F0E87
:101DF000E926000EEA22580EEE6E020EEF6E100E6D
:101E0000DBCFE9FFE828DBCFEAFFEF50010A01E072
:101E100016D15FEC28F0100EDBCFE9FFE828DBCF0E
:101E2000EAFF140EE926000EEA22E9CF00F0EACF1D
:101E300001F00101F02BF123F223F32300C0E9FFAD
:101E400001C0EAFFF0C1EEFFF1C1EEFFF2C1EEFF0B
:101E5000F3C1EFFF100EDBCFE9FFE828DBCFEAFF8D
:101E6000180EE926000EEA22E9CF00F0EACF01F0D1
:101E7000DE2ADE22DE22DF22DDCF05F0DDCF04F018
:101E8000DDCF03F0DFCF02F000C0E9FF01C0EAFFC1
:101E900002C0EEFF03C0EEFF04C0EEFF05C0EFFF7F
:101EA000100EDBCFE9FFE828DBCFEAFF140EE926AE
:101EB000000EEA22EECF00F0EECF01F0EECF02F0FE
:101EC000EECF03F0040E00C0DBFF050E01C0DBFF08
:101ED000060E02C0DBFF070E03C0DBFF100EDBCFD8
:101EE000E9FFE828DBCFEAFF140EE926000EEA221C
:101EF000EE2AEE22EE22EF22FA0EDBCFE9FFE828EF
:101F0000DBCFEAFF0D0EE926000EEA22EFB2010E4A
:101F1000E8504EE00A0EE66EE66AFC0EDBCF00F0FB
:101F2000E828DBCF01F000C0E6FF01C0E6FF100E9D
:101F3000DBCFE9FFE828DBCFEAFFEE52E9CF02F082
:101F4000EACF03F002C0E6FF03C0E6FF10EC38F072
:101F5000060EE15E100EDBCFE9FFE828DBCFEAFFDB
:101F60000D0EE926000EEA22E9CF00F0EACF01F0DB
:101F7000FA0EDBCFE9FFE828DBCFEAFFEECF02F075
:101F8000EECF03F000C0E9FF01C0EAFF02C0EEFFA0
:101F900003C0EDFF120EE76EE7CFDBFF100EDBCFC5
:101FA000E9FFE828DBCFEAFF020EEF6EFAEF13F04D
:101FB000040EE76E120EE7CFDBFFDECF00F0DDCFC1
:101FC00001F0020EDBCF02F0030EDBCF03F0040EB4
:101FD00000C0DBFF050E01C0DBFF060E02C0DBFF09
:101FE000070E03C0DBFFFA0EDBCFE9FFE828DBCFEB
:101FF000EAFF040EE926000EEA22EECF00F0EECF53
:1020000001F0EECF02F0EECF03F000C0DEFF01C022
:10201000DDFF020E02C0DBFF030E03C0DBFF100E6C
:10202000DBCFE9FFE828DBCFEAFFEE52060EE92618
:10203000000EEA22EE6AEE6AEE6AEF6ADBD3FA0E6F
:10204000DBCFE9FFE828DBCFEAFF0D0EE926000E23
:10205000EA22EFB4010EE85012E05FEC28F0100E17
:10206000DBCF00F0E828DBCF01F000C0E6FF01C0C5
:10207000E6FF64EC0DF0E550E55056EF14F0040E69
:10208000DBCF00F0050EDBCF01F0060EDBCF02F058
:10209000070EDBCF03F0FA0EDBCFE9FFE828DBCF3A
:1020A000EAFF080EE926000EEA22EECF04F0EECF9A
:1020B00005F0EECF06F0EECF07F00050045C01E033
:1020C00097D30150055801E093D30250065801E020
:1020D0008FD30350075801E08BD3100EDBCFE9FFFD
:1020E000E828DBCFEAFFEF50020A01E078D0FA0ED1
:1020F000DBCFE9FFE828DBCFEAFF0D0EE926000E73
:10210000EA22EFB8010EE85001E172D3100EDBCFE6
:10211000E9FFE828DBCFEAFF180EE926000EEA22E5
:10212000E9CF00F0EACF01F0DECF02F0DDCF03F01F
:10213000020EDBCF04F0030EDBCF05F000C0E9FF99
:1021400001C0EAFF02C0EEFF03C0EEFF04C0EEFFD5
:1021500005C0EFFF100EDBCFE9FFE828DBCFEAFF79
:102160001C0EE926000EEA22EF6A100EDBCFE9FF13
:10217000E828DBCFEAFF1D0EE926000EEA22E9CFB0
:1021800000F0EACF01F000C0E6FF01C0E6FF74EC0A
:102190003AF0F4CF03F0F3CF02F0E550E5CF01F0D1
:1021A000E7CF00F000C0E9FF01C0EAFF02C0EEFF88
:1021B00003C0EDFF100EDBCFE9FFE828DBCFEAFF1D
:1021C000040EEF6EF80EDBCF00F0E828DBCF01F055
:1021D00000500008000E015401E30AD39ED0100EF7
:1021E000DBCFE9FFE828DBCFEAFFEF50030A01E08D
:1021F000C7D0FA0EDBCFE9FFE828DBCFEAFF0D0EF0
:10220000E926000EEA22EFB2010EE85001E1F0D219
:10221000100EDBCFE9FFE828DBCFEAFF180EE92636
:10222000000EEA22E9CF00F0EACF01F0DE2ADE223A
:10223000DE22DF22DDCF05F0DDCF04F0DDCF03F0BD
:10224000DFCF02F000C0E9FF01C0EAFF02C0EEFFED
:1022500003C0EEFF04C0EEFF05C0EFFFFA0EDBCFB8
:10226000E9FFE828DBCFEAFF0D0EE926000EEA229F
:10227000EFB8010EE8500EE0100EE76E120EE7CF39
:10228000DBFF100EDBCFE9FFE828DBCFEAFF040E0F
:10229000EF6E37D0120EE76EE7CFDBFF100EDBCF0D
:1022A000E9FFE828DBCFEAFF020EEF6E100EDBCF6E
:1022B000E9FFE828DBCFEAFF140EE926000EEA2248
:1022C000E9CF00F0EACF01F0040ED926000EDE2A95
:1022D000DE22DE22DF22DDCF05F0DDCF04F0DDCF10
:1022E00003F0DFCF02F0040ED95E00C0E9FF01C0A9
:1022F000EAFF02C0EEFF03C0EEFF04C0EEFF05C020
:10230000EFFFF80EDBCF00F0E828DBCF01F0005044
:102310000008000E015401E36BD2100EDBCFE9FF81
:10232000E828DBCFEAFF210EE926000EEA22EF863D
:10233000100EDBCFE9FFE828DBCFEAFF120EE9261B
:10234000000EEA22E9CF00F0EACF01F0F80EDBCF71
:1023500002F0E828DBCF03F000C0E9FF01C0EAFF8C
:1023600002C0EEFF03C0EDFF100EDBCFE9FFE8284F
:10237000DBCFEAFF210EE926000EEA22EF843AD2F3
:10238000FA0EDBCFE9FFE828DBCFEAFF040EE926EF
:10239000000EEA22EECF00F0EECF01F0EECF02F019
:1023A000EECF03F0100EDBCFE9FFE828DBCFEAFF2A
:1023B000180EE926000EEA22EECF04F0EECF05F06B
:1023C000EECF06F0EECF07F00050045C08E10150BC
:1023D000055805E10250065802E10350075803E092
:1023E0005FEC28F063D2100EDBCFE9FFE828DBCFEB
:1023F000EAFF180EE926000EEA22E9CF00F0EACF44
:1024000001F0DECF02F0DDCF03F0020EDBCF04F0EF
:10241000030EDBCF05F000C0E9FF01C0EAFF02C0F8
:10242000EEFF03C0EEFF04C0EEFF05C0EFFF100E8D
:10243000DBCFE9FFE828DBCFEAFFEF50040A01E039
:102440003ED1FA0EDBCFE9FFE828DBCFEAFF0D0E25
:10245000E926000EEA22EFB8010EE85032E0100E35
:10246000DBCFE9FFE828DBCFEAFF0F0EE926000EFD
:10247000EA22EF50FF0A25E0100EDBCFE9FFE82843
:10248000DBCFEAFF0F0EE926000EEA22EF50E66EE0
:10249000E9EC28F0E550100EDBCFE9FFE828DBCFB0
:1024A000EAFF0F0EE926000EEA22EF68100EDBCFDE
:1024B000E9FFE828DBCFEAFF210EE926000EEA2239
:1024C000EF82FA0EDBCFE9FFE828DBCFEAFF0D0E43
:1024D000E926000EEA22EF50010BE8504FE0110E02
:1024E000E76E120EE7CFDBFF100EDBCFE9FFE82827
:1024F000DBCFEAFF140EE926000EEA22EECF00F051
:10250000EECF01F0EDCF02F0ED50000EEE2AEE22FC
:10251000EE22EF22040E00C0DBFF050E01C0DBFF40
:10252000060E02C0DBFF070E03C0DBFF100EDBCF81
:10253000E9FFE828DBCFEAFF180EE926000EEA22C1
:10254000EE2AEE22EE22EF22EDCF03F0EDCF02F0E5
:10255000EDCF01F0EFCF00F000C0DEFF01C0DDFFE6
:10256000020E02C0DBFF030E03C0DBFF100EDBCF49
:10257000E9FFE828DBCFEAFF0A0EEF6EF80EDBCFAB
:1025800000F0E828DBCF01F000500008000E0154F5
:1025900001E32ED1100EDBCFE9FFE828DBCFEAFF05
:1025A000210EE926000EEA22EFB6010EE86638D0C9
:1025B000100EDBCFE9FFE828DBCFEAFF210EE9268A
:1025C000000EEA22EF86100EDBCFE9FFE828DBCF12
:1025D000EAFF120EE926000EEA22E9CF00F0EACF68
:1025E00001F0F80EDBCF02F0E828DBCF03F000C0EB
:1025F000E9FF01C0EAFF02C0EEFF03C0EDFF100ECD
:10260000DBCFE9FFE828DBCFEAFF210EE926000E49
:10261000EA22EF84100EE76E120EE7CFDBFFEAD05E
:10262000120EDB6A100EDBCFE9FFE828DBCFEAFFF2
:10263000140EE926000EEA22E9CF00F0EACF01F0FD
:102640000C0EDBCF02F00D0EDBCF03F00E0EDBCF56
:1026500004F00F0EDBCF05F000C0E9FF01C0EAFF78
:1026600002C0EEFF03C0EEFF04C0EEFF05C0EFFFA7
:10267000100EDBCFE9FFE828DBCFEAFF180EE926D2
:10268000000EEA22E9CF00F0EACF01F0080EDBCF1E
:1026900002F0090EDBCF03F00A0EDBCF04F00B0EC5
:1026A000DBCF05F000C0E9FF01C0EAFF02C0EEFF8A
:1026B00003C0EEFF04C0EEFF05C0EFFF99D0100E7F
:1026C000DBCFE9FFE828DBCFEAFFEF500A0A12E18F
:1026D0005FEC28F0FA0EDBCFE9FFE828DBCFEAFF5A
:1026E0000D0EE926000EEA22EFB8010EE85001E1D6
:1026F00081D06FD0100EDBCFE9FFE828DBCFEAFFF7
:10270000EF50050A4DE15FEC28F0FA0EDBCFE9FF50
:10271000E828DBCFEAFF0D0EE926000EEA22EF5093
:10272000010BE85067E0100EE76E120EE7CFDBFFFB
:10273000100EDBCFE9FFE828DBCFEAFF180EE92611
:10274000000EEA22EE2AEE22EE22EF22EDCF03F077
:10275000EDCF02F0EDCF01F0EFCF00F000C0DEFFD3
:1027600001C0DDFF020E02C0DBFF030E03C0DBFF72
:10277000FA0EDBCFE9FFE828DBCFEAFF0D0EE926F2
:10278000000EEA22EFB8010EE85001E022D0100E50
:10279000DBCFE9FFE828DBCFEAFF060EEF6E2AD099
:1027A000100EDBCFE9FFE828DBCFEAFFEF50060A87
:1027B00021E15FEC28F0FA0EDBCFE9FFE828DBCF60
:1027C000EAFF0D0EE926000EEA22EFB8010EE850EE
:1027D00011E0100EDBCF00F0E828DBCF01F000C0E5
:1027E000E6FF01C0E6FF64EC0DF0E550E55002D0D5
:1027F0005FEC28F0120EDB50000858E2E66AE66A49
:10280000E668120EDB50E66EDECF00F0DDCF01F0A1
:10281000020EDBCF02F0030EDBCF03F000C0E6FFB9
:1028200001C0E6FF02C0E6FF03C0E6FF040EDBCFF7
:1028300004F0050EDBCF05F0060EDBCF06F0070E29
:10284000DBCF07F004C0E6FF05C0E6FF06C0E6FFE9
:1028500007C0E6FFFA0EDBCFE9FFE828DBCFEAFF8F
:10286000EECF08F0EECF09F008C0E6FF09C0E6FFA2
:10287000FA0EDBCFE9FFE828DBCFEAFFEE52EE529B
:10288000EECF0AF0EECF0BF00AC0E6FF0BC0E6FF7A
:10289000FC0EDBCF0CF0E828DBCF0DF00CC0E6FF20
:1028A0000DC0E6FFFAEC07F0120EE15E140EE15ED9
:0628B000E7CFD9FF120082
:0A28B600DACFE4FFE652E9CFE6FFB7
:1028C000EACFE6FF000EE96E000EEA6E160EE8048F
:1028D00003E3EECFE6FFFBD779EC3AF0A8EC26F065
:1028E000E552150EE96E000EEA6E160EE80403E3DB
:1028F000E5CFEDFFFBD7E5CFEAFFE5CFE9FFE5CF79
:10290000DAFF1100D9CFE6FFE1CFD9FFACB201D099
:10291000FDD7FE0EDB50AD6EE552E7CFD9FF1200BA
:10292000D9CFE6FFE1CFD9FF010EE126FD0EDBCFC7
:10293000E9FFDB2AFE0EDBCFEAFF01E1DB2AEECF67
:1029400000F0000E00C0DBFFDB50E85006E0DF5077
:10295000E66E82EC14F0E550E9D7020EE15EE7CFB7
:10296000D9FF1200F86A86EC17F06AEC3AF03CECFA
:1029700032F0A7EC17F081BA0FD0C00EE66E38EC3B
:1029800036F0E550070EE66E6E0EE66EA9EC36F0F8
:10299000E550E550BFEC1AF0E5EC34F043EC1CF0E8
:1029A000EEEC34F086EC1CF014EC16F00001E4516F
:1029B000E35DF6E0010EE66E000E006E020E016EA3
:1029C00000C0E6FF01C0E6FF01EC15F0E550E55060
:1029D000E550E4C0E3F0020118A1E2D7CE0EE66EA6
:1029E00038EC36F0E5500A0E0001E35D03E2E351F6
:1029F000300F02D0E351410FE66ECEEC36F0E550D9
:102A0000CFD7D9CFE6FFE1CFD9FF080EE126FC0EE4
:102A1000DB5012E0C00EE66E38EC36F0E550160ED4
:102A2000E66E6E0EE66EA9EC36F0E550E550C00E8F
:102A3000E66E38EC36F0E550D9CF00F0DACF01F091
:102A400000C0E6FF01C0E6FFFD0EDBCFE9FFE8288E
:102A5000DBCFEAFFEECF02F0036A02C0E6FF03C05D
:102A6000E6FF4BEC34F0040EE15EFC0EDB5011E0AF
:102A7000D9CF00F0DACF01F000C0E6FF01C0E6FFD9
:102A800085EC36F0E550E5502E0EE66ECEEC36F0D5
:102A900010D0D9CF00F0DACF01F000C0E6FF01C0BE
:102AA000E6FF90EC14F0E550E5502E0EE66E82EC59
:102AB00014F0E550D9CF00F0DACF01F000C0E6FF06
:102AC00001C0E6FFFD0EDBCFE9FFE828DBCFEAFF20
:102AD000EE52EECF02F0036A02C0E6FF03C0E6FF4B
:102AE0004BEC34F0040EE15EFC0EDB5011E0D9CF6C
:102AF00000F0DACF01F000C0E6FF01C0E6FF85EC90
:102B000036F0E550E5502E0EE66ECEEC36F010D0E5
:102B1000D9CF00F0DACF01F000C0E6FF01C0E6FF38
:102B200090EC14F0E550E5502E0EE66E82EC14F0B9
:102B3000E550D9CF00F0DACF01F000C0E6FF01C0C8
:102B4000E6FFFD0EDBCFE9FFE828DBCFEAFFEE5220
:102B5000EE52EECF02F0036A02C0E6FF03C0E6FFCA
:102B60004BEC34F0040EE15EFC0EDB5011E0D9CFEB
:102B700000F0DACF01F000C0E6FF01C0E6FF85EC0F
:102B800036F0E550E5502E0EE66ECEEC36F010D065
:102B9000D9CF00F0DACF01F000C0E6FF01C0E6FFB8
:102BA00090EC14F0E550E5502E0EE66E82EC14F039
:102BB000E550D9CF00F0DACF01F000C0E6FF01C048
:102BC000E6FFFD0EDBCFE9FFE828DBCFEAFFEE52A0
:102BD000EE52EE52EECF02F0036A02C0E6FF03C0EF
:102BE000E6FF4BEC34F0040EE15EFC0EDB500BE034
:102BF000D9CF00F0DACF01F000C0E6FF01C0E6FF58
:102C000085EC36F00AD0D9CF00F0DACF01F000C061
:102C1000E6FF01C0E6FF90EC14F0E550E550090E28
:102C2000E15EE7CFD9FF1200D9CFE6FFE1CFD9FFB0
:102C3000020EE126810EC26E640EDF6EDF50DF06EB
:102C4000E85001E0FBD7C284C2A401D0FDD7C3CFB6
:102C5000DFFF010EC4CFDBFF190EE66E020EE66E3B
:102C6000000EDBCF00F0E828DBCF01F000C0E6FF6C
:102C700001C0E6FF4BEC34F0040EE15E840EC16E41
:102C8000890EC26E640EDF6EDF50DF06E85001E091
:102C9000FBD7C284C2A401D0FDD7C3CFDFFF010E92
:102CA000C4CFDBFF210EE66E020EE66E000EDBCF18
:102CB00000F0E828DBCF01F000C0E6FF01C0E6FF2E
:102CC0004BEC34F0040EE15E8E0EC16E030EE15E3D
:102CD000E7CFD9FF1200D9CFE6FFE1CFD9FF020E2F
:102CE000E126FD0EDBCFE9FFE828DBCFEAFFEE505F
:102CF000EDCFEAFFE96EEF50D00F006E00C0DFFFAE
:102D0000DF50010A48E0010A01E024D0FD0EDBCFCC
:102D1000E9FFE828DBCFEAFFEE52EE52EE50EDCFAE
:102D2000EAFFE96EEF50D00F006E010E00C0DBFF2E
:102D3000DB50010A06E0010A01E005D00F018976A7
:102D400002D00F0189740D0EE66EE66A270E006E42
:102D50006E0E06D00A0EE66EE66A340E006E6E0E39
:102D6000016E0001026B00C0E6FF01C0E6FF02C079
:102D7000E6FFFD0EDBCFE9FFE828DBCFEAFFEECF71
:102D800003F0EECF04F003C0E6FF04C0E6FF3BEC27
:102D900038F0070EE15E030EE15EE7CFD9FF1200C7
:102DA000D9CFE6FFE1CFD9FFFE0EDB50040A01E1E7
:102DB00095D0070A4DE0010A0BE0030A06E0010A7C
:102DC00001E09ED089A68CD093D089A489D090D0E0
:102DD000D9CFE9FFDACFEAFFFC0EE926EE5007E192
:102DE000ED5005E1FC0ED926DE6ADD6AD95EFA0EE9
:102DF000DBCF00F0E828DBCF01F0D9CFE9FFDACF55
:102E0000EAFFFC0EE926EF50EA6A190FE96E020E9E
:102E1000EA22EF5000C0E9FF01C0EAFFEF6ED9CF10
:102E2000E9FFDACFEAFFFC0EE926EF50EA6A190F54
:102E3000E96E020EEA22EF5001E162D0FC0EDBCF18
:102E400000F0DB2AFD0EDBCF01F041E1DB2A3FD0B1
:102E5000D9CFE9FFDACFEAFFFC0EE926EE5007E111
:102E6000ED5005E1FC0ED926DE6ADD6AD95EFA0E68
:102E7000DBCF00F0E828DBCF01F0D9CFE9FFDACFD4
:102E8000EAFFFC0EE926EF50EA6A210FE96E020E16
:102E9000EA22EF5000C0E9FF01C0EAFFEF6ED9CF90
:102EA000E9FFDACFEAFFFC0EE926EF50EA6A210FCC
:102EB000E96E020EEA22EF5001E122D0FC0EDBCFD8
:102EC00000F0DB2AFD0EDBCF01F001E1DB2AFC0E76
:102ED000DBCFF3FFE828DBCFF4FF14D081AA08D0C2
:102EE000FA0EDBCFE9FFE828DBCFEAFF310E07D08F
:102EF000FA0EDBCFE9FFE828DBCFEAFF300EEF6EFA
:102F0000F368F468E552E7CFD9FF12008E0EC16E68
:102F1000030E926E809A89848986F19EF1EC35F0D9
:102F2000800EE66E38EC36F0E550F80EE66E6D0E6B
:102F3000E66EA9EC36F0E550E550200EAC6E900E32
:102F4000AB6E0F0EAF6ED56AF28EF28C1200D9CF37
:102F5000E6FFE1CFD9FF030EE12602010A0E006F62
:102F6000016F050E026F0F0E036F0A690B690C6982
:102F70000D6B0A0E0E6F0F6F050E106F0F0E116F97
:102F8000046B040E056FA30E066F076B086B096BCD
:102F90001891D9CFE9FFDACFEAFF010EE926000E3A
:102FA000EE6E020EED6EE66AE66AA00EE66E16ECB6
:102FB0002FF0E550E550E550AEEC2FF0F3CF00F0E8
:102FC00000C0DFFFBBEC2FF0DF50550A2DE1010EF2
:102FD000E66EE66AA00EE66E16EC2FF0E550E550C0
:102FE000E550DF6ADF50E70F1CE2010EDBCF00F097
:102FF000DB2A020EDBCF01F001E1DB2A00C0E6FF95
:1030000001C0E6FFAEEC2FF0E550E5CF01F0E7CFD1
:1030100000F0F35000C0E9FF01C0EAFFEF6EDF2AC5
:10302000E1D7BBEC2FF002D01BEC18F0040EE15EF0
:10303000E7CFD9FF1200D9CFE6FFE1CFD9FF030ECA
:10304000E126D9CFE9FFDACFEAFF010EE926000E2B
:10305000EE6E020EED6EE66AE66AA00EE66EAEEC6D
:103060002EF0E550E550E550550EE66E72EC2FF06F
:10307000E550DF6ADF50E70F10E2010EDBCFE9FF1A
:10308000DB2A020EDBCFEAFF01E1DB2AEF50E66E1E
:1030900072EC2FF0E550DF2AEDD79EEC2FF0040EF6
:1030A000E15EE7CFD9FF1200D9CFE6FFE1CFD9FF2C
:1030B000010EE126FD0EDBCFF6FFDB2AFE0EDBCF95
:1030C000F7FF01E1DB2A0A00F5CF00F0000E00C097
:1030D000DBFFDB50E85006E0DF50E66E82EC14F0D8
:1030E000E550E8D7020EE15EE7CFD9FF1200D9CF55
:1030F000E6FFE1CFD9FF020EE126010EDB6A9EBAA0
:1031000001D0FDD7AECFDFFFDF500D0AD87403E149
:10311000DF500A0AD87401E01FD0010EDB2AFD0E31
:10312000DBCF00F0DB2AFE0EDBCF01F001E1DB2A72
:10313000DF5000C0E9FF01C0EAFFEF6EFD0EDBCFFC
:10314000E9FFE828DBCFEAFFEF6AFC0EDBCFE9FFFF
:10315000DB06E950E866D3D7010EDB50F36E030EB1
:10316000E15EE7CFD9FF1200D9CFE6FFE1CFD9FF6B
:10317000040EE126FD0EDBCF00F0E828DBCF01F0E6
:10318000010E00C0DBFF020E01C0DBFF030EDB6A95
:10319000FD0EDBCFE9FFE828DBCFEAFFEECF00F042
:1031A000000E00C0DBFFDB50E85062E0DF502E0A6B
:1031B00050E1FD0EDBCFE9FFDB2AFE0EDBCFEAFF9D
:1031C00001E1DB2AEF6AFB0EDBCFE9FFE828DBCF6A
:1031D000EAFFE9CF02F0EACF03F0030EDBCFE9FF0D
:1031E000DB2AE950016A0224006E0350012200C06C
:1031F000E6FF01C0E6FF02C0E6FF03C0E6FF010EE6
:10320000DBCF04F0E828DBCF05F004C0E6FF05C003
:10321000E6FFD6EC33F0E550E550E550E5CF03F09E
:10322000E5CF02F0E5CF01F0E7CF00F0F35000C0AA
:10323000E9FF01C0EAFFEF6EFD0EDBCF00F0E828EA
:10324000DBCF01F0010E00C0DBFF020E01C0DBFF8F
:1032500009D0DF50D00F01E203D0DF50390802E27D
:10326000F36A45D0FD0EDB2A93E1FE0EDB2A90D7F0
:10327000FB0EDBCFE9FFE828DBCFEAFFE9CF02F066
:10328000EACF03F0030EDB50016A0224006E035004
:10329000012200C0E6FF01C0E6FF02C0E6FF03C056
:1032A000E6FF010EDBCF04F0E828DBCF05F004C019
:1032B000E6FF05C0E6FFD6EC33F0E550E550E550FB
:1032C000E5CF03F0E5CF02F0E5CF01F0E7CF00F066
:1032D000F35000C0E9FF01C0EAFFEF6E030EDB50C0
:1032E000030A01E102D0000E01D0010EF36E050EBB
:1032F000E15EE7CFD9FF1200D9CFE6FFE1CFD9FFDA
:10330000010EE1269EBA01D0FDD7AECFDFFFDF5020
:10331000CF0F01E206D0DF50C70F01E302D0DF502C
:1033200001D0390EF36E020EE15EE7CFD9FF120035
:10333000D9CFE6FFE1CFD9FF1A0EE1260D0EE66EDA
:1033400082EC14F0E5500A0EE66E82EC14F0E550C3
:10335000FE0EDB50D00FFF0F020DF3CFE9FFF4CFCD
:10336000EAFFE50EE926000EEA22EECF00F0EECFEE
:1033700001F000C0E6FF01C0E6FF54EC18F0E55094
:10338000E550FE0EDB50380A01E1F2D00F0A01E1F0
:10339000ECD0010A01E1E6D0030A01E1E0D0010A24
:1033A00060E0070A5AE0010A54E0030A01E0E2D0B3
:1033B000D9CF00F0DACF01F000C0E6FF01C0E6FF90
:1033C00012C2E6FF13C2E6FF4BEC34F0040EE15EDE
:1033D000D9CF00F0DACF01F000C0E6FF01C0E6FF70
:1033E00090EC14F0E550E550290EE66E82EC14F0F6
:1033F000E5503A0EE66E82EC14F0E550200EE66ED3
:1034000082EC14F0E550140EE66ED9CF00F0DACF5E
:1034100001F000C0E6FF01C0E6FF77EC18F0E550D0
:10342000E550E550F3506DE0D9CF00F0DACF01F070
:1034300000C0E6FF01C0E6FFD6EC33F0F4CF13F294
:10344000F3CF12F2E550E55013C208F212C209F2AE
:1034500091D0000E006E020E07D00E0E006E020E0E
:1034600003D00A0E006E020E016E180E00C0DBFFC4
:10347000190E01C0DBFFE66A180EDBCF00F0E8286A
:10348000DBCF01F000C0E6FF01C0E6FF01EC15F064
:10349000E550E550E550290EE66E82EC14F0E5505B
:1034A0003A0EE66E82EC14F0E550200EE66E82ECE9
:1034B00014F0E550140EE66ED9CF00F0DACF01F02B
:1034C00000C0E6FF01C0E6FF77EC18F0E550E550DC
:1034D000E550D9CF00F0DACF01F0140E002600C07D
:1034E000E6FF01C0E6FFD9CF02F0DACF03F002C059
:1034F000E6FF03C0E6FFB4EC18F0040EE15EF35003
:103500000BE1950EE66E6F0EE66E54EC18F0E5508A
:10351000E5509EBA2FD0FDD7180EDBCFE9FFE82883
:10352000DBCFEAFFE9CF00F0EACF01F0140EDBCFEA
:1035300002F0150EDBCF03F0160EDBCF04F0170EF2
:10354000DBCF05F000C0E9FF01C0EAFF02C0EEFFDB
:1035500003C0EEFF04C0EEFF05C0EFFF0BD0020179
:10356000188108D00201189105D0E3EC1AF002D0BE
:103570001BEC18F01B0EE15EE7CFD9FF1200D9CF8C
:10358000E6FFE1CFD9FF010EE1263E0EE66E6E0E9C
:10359000E66E54EC18F0E550E5507CEC19F0F3CFF2
:1035A00000F000C0DFFFDF50390A05E0DF50E66EB3
:1035B00098EC19F0E550DF50380AE7E1020EE15EC1
:1035C000E7CFD9FF1200D9CFE6FFE1CFD9FF0E0E2A
:1035D000E126DF6A040EDB6A66EC33F0F4CF01F01B
:1035E000F3CF00F0020E00C0DBFF030E01C0DBFFD3
:1035F000070ED926DE6A040EDD6E070ED95E74EC66
:103600003AF0F4CF01F0F3CF00F0090E00C0DBFF79
:103610000A0E01C0DBFF74EC3AF0F4CF01F0F3CFF7
:1036200000F00B0E00C0DBFF0C0E01C0DBFF0B0E29
:10363000DBCF04F0E828DBCF05F0090EDBCF06F086
:10364000E828DBCF07F00650045C0750055801E27C
:1036500002D0000E01D0010E026E036A02BE0368A2
:10366000025003E1035001E11BD00A680B68090E08
:10367000DBCF0CF0E828DBCF0DF00C500A5C086EB5
:103680000D500B58096E0B0EDBCF0EF0E828DBCF88
:103690000FF00E500824006E0F500920016E20D04C
:1036A0000B0EDBCF12F0E828DBCF13F0090EDBCFD7
:1036B00014F0E828DBCF15F01450125C106E155092
:1036C0001358116E050E105C000E115801E302D064
:1036D000000E01D0010E006E0001016B00BF0169F8
:1036E000005001E1015013E074EC3AF0F4CF01F026
:1036F000F3CF00F0090E00C0DBFF0A0E01C0DBFFB4
:10370000150EE66E82EC14F0E5500F0189749EAA46
:1037100082D7040EDB5001E093D09EAAFAD70F01A6
:103720008974010EAECFDBFFDF50030A2DE0010AE2
:1037300028E0030A1EE0010EDB50010A02E1010E3F
:1037400021D0010EDB50040A0EE189840AEC33F02B
:10375000060EE66E82EC14F0E550010EE76E040EE4
:10376000E7CFDBFFD6D7150EE66E82EC14F0E550FE
:10377000D0D7060EE76EE7CFDBFF050EDB6A020E41
:1037800001D0030EDF6EC5D7050EDBCFE9FFDB2AC4
:10379000E950E76E070EDBCF00F0080EDBCF01F03B
:1037A000E7500026000E0122010EDB5000C0E9FFA9
:1037B00001C0EAFFEF6E050EDB508008AAE2020EA0
:1037C000DBCF00F0E828DBCF01F000C0E6FF01C04E
:1037D000E6FF6CEC33F0E550E550060EE76EE7CF00
:1037E000DBFF010EDB6A010EDB50800F15E2010EDC
:1037F000DB50E76E070EDBCFE9FF080EDBCFEAFFF9
:10380000E750E926000EEA22EF50E66E9DEC33F019
:10381000E550010EDB2AE7D7C5EC33F0F4CF01F019
:10382000F3CF00F0020E00C0DBFF030E01C0DBFF90
:10383000060EDB50E66E82EC14F0E550DF6A69D7C5
:103840000D0EDB680D0EDBCFE9FFDB06E950E8501B
:1038500001E0F8D7010EF36E0F0EE15EE7CFD9FF5E
:1038600012004C0EE66E86EC3AF0E5501200150E92
:10387000E66E86EC3AF0E5501200330EE66EA2ECEE
:063880003AF0E5501200D1
:0A388600D9CFE6FFE1CFD9FF010E14
:10389000E126DF6ADF50FB0F34E2DF500A0DF3CF81
:1038A000E9FFF4CFEAFF800EE926000EEA22E9CF15
:1038B00000F0EACF01F000C0E6FF01C0E6FF500EC5
:1038C000E66EE66A07EC01F0E550E550E550E5CF1D
:1038D00001F0E7CF00F0F35000C0E9FF01C0EAFFBC
:1038E000EF6EDF500A0DF3CFE9FFF4CFEAFF800E51
:1038F000E926000EEA22EE52EE52EE52EF6ADF2A7D
:10390000C9D7020EE15EE7CFD9FF1200D9CFE6FF9B
:10391000E1CFD9FF010EE126DF6ADF50FB0F07E29E
:10392000DF50E66E9CEC1CF0E550DF2AF6D7020E65
:10393000E15EE7CFD9FF1200D9CFE6FFE1CFD9FF93
:10394000650EE126FE0EDB500A0DF3CF00F0F4CF3A
:1039500001F0800E0026000E0122610E00C0DBFF88
:10396000620E01C0DBFF010EE76E540EE7CFDBFFF6
:10397000540EDB5001E117D3540EDB6A610EDBCF2E
:10398000E9FFE828DBCFEAFFEF50E66E9FEC01F09D
:10399000E550F3500BE1610EDBCFE9FFE828DBCF08
:1039A000EAFFEE52EE52EE52EF6AFDD2610EDBCF2D
:1039B000E9FFE828DBCFEAFFEE52EE52EE52EF507D
:1039C000090A01E1BDD2080A01E184D20A0A01E133
:1039D000B2D1090A01E155D1020A01E0C9D7610E4D
:1039E000DBCFE9FFE828DBCFEAFFEF50E66EFEEC25
:1039F00005F0E550F350BCE0010EE76E540EE7CF42
:103A0000DBFF520ED926DE6ADD6AD95E520EDBCFAD
:103A100000F0E828DBCF01F0500E005C000E0158EA
:103A200001E32FD000C0E6FF01C0E6FFD9CF04F0CC
:103A3000DACF05F0520EDBCF06F0DB2A530EDBCFD8
:103A400007F001E1DB2A06500424026E075005202E
:103A5000036E02C0E6FF03C0E6FF610EDBCFE9FFA5
:103A6000E828DBCFEAFFEF50E66E72EC05F0E55098
:103A7000E550E550E550E5CF01F0E7CF00F0F35019
:103A8000C5E1D9CF00F0DACF01F0520EDBCF02F062
:103A9000E828DBCF03F002500024E96E0350012038
:103AA000EA6EEF6A610EDBCFE9FFE828DBCFEAFFC1
:103AB000EF50E66EC9EC04F0E550610EDBCFE9FF94
:103AC000E828DBCFEAFFEE52EE52EE52020EEF6E26
:103AD000050EE76E5F0EE7CFDBFF610EDBCFE9FF80
:103AE000E828DBCFEAFF090EE926000EEA22E9CF3B
:103AF00001F0EACF02F001C0E6FF02C0E6FFD9CF35
:103B000003F0DACF04F05F0E032603C0E6FF04C023
:103B1000E6FFD9CF05F0DACF06F0550E052605C031
:103B2000E6FF06C0E6FFD9CF07F0DACF08F007C0FE
:103B3000E6FF08C0E6FF74EC21F0080EE15EF3CF6B
:103B400000F0510E00C0DBFFDB50E86611D75F0EBE
:103B5000DB5001081EE25F0EDB50E66ED9CF00F0AD
:103B6000DACF01F0550E002600C0E6FF01C0E6FFE7
:103B70006BEC16F0E550E550E550610EDBCFE9FF48
:103B8000E828DBCFEAFF090EE926000EEA22030E41
:103B9000EF6E610EDBCFE9FFE828DBCFEAFFEE52E4
:103BA000E9CF00F0EACF01F000C0E6FF01C0E6FF78
:103BB000550EDBCF04F0E828DBCF05F004C0E6FFAC
:103BC00005C0E6FF47EC32F0F4CF03F0F3CF02F08C
:103BD000E550E550E550E5CF01F0E7CF00F000C03B
:103BE000E9FF01C0EAFF02C0EEFF03C0EDFF610E76
:103BF000DBCFE9FFE828DBCFEAFFEE52EECF00F0A3
:103C0000EECF01F0FF0E005C0FE1FF0E01580CE15A
:103C1000610EDBCFE9FFE828DBCFEAFF080EE926DB
:103C2000000EEA22EF6A17D0610EDBCFE9FFE82829
:103C3000DBCFEAFFEE52EE5019E1ED5017E1610ED5
:103C4000DBCFE9FFE828DBCFEAFF080EE926000E0C
:103C5000EA22030EEF6E610EDBCFE9FFE828DBCF2F
:103C6000EAFFEE52EE52EE52020E9BD1610EDBCF16
:103C7000E9FFE828DBCFEAFFEE52EE52EE520B0EE0
:103C800090D1610EDBCFE9FFE828DBCFEAFFEF50F0
:103C9000E66EC1EC03F0E550F35001E169D6610E28
:103CA000DBCFE9FFE828DBCFEAFF080EE926000EAC
:103CB000EA22EF50020DF3CFE9FFF4CFEAFF290E1D
:103CC000E926020EEA22EECF00F0EECF01F0630EFD
:103CD00000C0DBFF640E01C0DBFF630EDBCFF6FF2D
:103CE000DB2A640EDBCFF7FF01E1DB2A0A00F5CF08
:103CF00000F0600E00C0DBFFDB50E85010E0600E0B
:103D0000DB50E66E610EDBCFE9FFE828DBCFEAFF90
:103D1000EF50E66EF1EC03F0E550E550DED7610EB2
:103D2000DBCFE9FFE828DBCFEAFFEF50E66E74EC6B
:103D300002F0E550FAD0610EDBCFE9FFE828DBCFD7
:103D4000EAFFEF50E66EC1EC03F0E550F35001E1FD
:103D50000FD6010EE76E540EE7CFDBFF600EDB6A75
:103D6000600EDB50E10F1AE2600EDBCFF6FFF76A60
:103D7000640EF626730EF7220800F550E66E610E0B
:103D8000DBCFE9FFE828DBCFEAFFEF50E66EF1EC8E
:103D900003F0E550E550600EDB2AE2D7610EDBCF81
:103DA000E9FFE828DBCFEAFF090EE926000EEA2248
:103DB000EF50140DF3CFF6FFF4CFF7FFD80EF62631
:103DC000720EF722F6CF00F0F7CF01F0630E00C0BD
:103DD000DBFF640E01C0DBFF630EDBCFF6FFDB2AE7
:103DE000640EDBCFF7FF01E1DB2A0A00F5CF00F01C
:103DF000600E00C0DBFFDB50E85010E0600EDB50CF
:103E0000E66E610EDBCFE9FFE828DBCFEAFFEF507B
:103E1000E66EF1EC03F0E550E550DED7600EDB6AAC
:103E2000600EDB50FC0F1AE2600EDBCFF6FFF76A84
:103E3000840EF626730EF7220800F550E66E610E2A
:103E4000DBCFE9FFE828DBCFEAFFEF50E66EF1ECCD
:103E500003F0E550E550600EDB2AE2D7610EDBCFC0
:103E6000E9FFE828DBCFEAFF090EE926000EEA2287
:103E7000EF50030A0DE1610EDBCFE9FFE828DBCF4D
:103E8000EAFF070EE926000EEA22010EEF6E0BD0C4
:103E9000610EDBCFE9FFE828DBCFEAFF070EE9265A
:103EA000000EEA22EF6A610EDBCFE9FFE828DBCFE4
:103EB000EAFF040EE926000EEA22030EEF6E610E01
:103EC000DBCFE9FFE828DBCFEAFFEE52EE52EE52FD
:103ED000010E67D0610EDBCFE9FFE828DBCFEAFFF8
:103EE000EF50E66EFEEC05F0E550F3500BE0610E8E
:103EF000DBCFE9FFE828DBCFEAFFEF50E66EC9EC45
:103F000004F0E550610EDBCF00F0E828DBCF01F0D4
:103F100000C0E6FF01C0E6FFD8EC1FF0E550E55019
:103F2000F35001E125D50AEC33F0610EDBCFE9FF58
:103F3000E828DBCFEAFFEE52EE52EE52090E31D006
:103F4000610EDBCFE9FFE828DBCFEAFFEF50E66E3A
:103F50009FEC01F0E550F35001E10AD5610EDBCF93
:103F6000E9FFE828DBCFEAFFEF50E66EC1EC03F093
:103F7000E550F35001E1FCD4610EDBCFE9FFE82806
:103F8000DBCFEAFFEF50E66EBAEC01F0E550610ED0
:103F9000DBCFE9FFE828DBCFEAFFEE52EE52EE522C
:103FA0000A0EEF6EE5D4660EE15EE7CFD9FF120090
:103FB000D9CFE6FFE1CFD9FF020EE126FD0EDBCF20
:103FC000E9FFE828DBCFEAFFEE52EECF00F0EECFBC
:103FD00001F000C0E6FF01C0E6FF11EC33F0E55050
:103FE000E550FD0EDBCFE9FFE828DBCFEAFFEF501D
:103FF000E66EC1EC03F0E550F35001E14DD1DF6A0C
:10400000FD0EDBCFE9FFE828DBCFEAFF040EE9264F
:10401000000EEA22EF50080A1EE037EC33F0F3CF2F
:1040200000F0010E00C0DBFF0201FF0E395D13E15D
:10403000FF0E3A5910E15FEC33F0FD0EDBCFE9FFE4
:10404000E828DBCFEAFFEF50E66E74EC02F0E550B3
:10405000010EF36E44D1FD0EDBCFE9FFE828DBCF84
:10406000EAFF070EE926000EEA22EF5001E106D131
:10407000FD0EDBCFE9FFE828DBCFEAFF040EE926DF
:10408000000EEA22EF50080A01E174D00E0A43E064
:10409000030A16E0060A01E0DFD0010EDB50250A14
:1040A0000CE1FD0EDBCFE9FFE828DBCFEAFF040ED1
:1040B000E926000EEA22050ECDD0010EDF6ECDD02E
:1040C000010EDB50250A03E1010EDF6EB8D0FD0EB4
:1040D000DBCFE9FFE828DBCFEAFF080EE926000E78
:1040E000EA22E9CF00F0EACF01F0010EDB50D00F59
:1040F0000F0BE83A00C0E9FF01C0EAFFEF6EFD0ECA
:10410000DBCFE9FFE828DBCFEAFF040EE926000E4B
:10411000EA22060E9FD0FD0EDBCFE9FFE828DBCFB9
:10412000EAFF080EE926000EEA22E9CF00F0EACF06
:1041300001F0010EDB50D00F00C0E9FF01C0EAFF23
:10414000EF12FD0EDBCFE9FFE828DBCFEAFF040E1C
:10415000E926000EEA22080EEF6EFD0EDBCFE9FF26
:10416000E828DBCFEAFF050EE926000EEA22EE6A18
:10417000EF6A73D0FD0EDBCFE9FFE828DBCFEAFF63
:10418000050EE926000EEA22E9CF00F0EACF01F0A1
:1041900000C0E6FF01C0E6FFD9CF04F0DACF05F09A
:1041A000010E042604C0E6FF05C0E6FFFD0EDBCFCE
:1041B000E9FFE828DBCFEAFF050EE926000EEA2238
:1041C000EECF06F0EECF07F006C0E6FF07C0E6FF31
:1041D000FD0EDBCFE9FFE828DBCFEAFF080EE9267A
:1041E000000EEA22EF50E66ED0EC16F0F4CF03F0AA
:1041F000F3CF02F0050EE15EE550E5CF01F0E7CF29
:1042000000F000C0E9FF01C0EAFF02C0EEFF03C0FA
:10421000EDFF010EDF6EFD0EDBCFE9FFE828DBCFFF
:10422000EAFF050EE926000EEA22EECF00F0EECFFF
:1042300001F0FF0E005C11E1FF0E01580EE1FD0ED2
:10424000DBCFE9FFE828DBCFEAFF040EE926000E0A
:10425000EA22030EEF6E01D0FFD7DF5001E1C1D695
:10426000010EDB50E66EFD0EDBCFE9FFE828DBCF69
:10427000EAFFEF50E66EF1EC03F0B1D6010EDB5031
:10428000E66EFD0EDBCFE9FFE828DBCFEAFFEF505B
:10429000E66EF1EC03F0A3D6FD0EDBCFE9FFE828D4
:1042A000DBCFEAFFEE52E9CF00F0EACF01F000C029
:1042B000E6FF01C0E6FF5FEC33F0F4CF03F0F3CF8D
:1042C00002F0E550E5CF01F0E7CF00F000C0E9FFD4
:1042D00001C0EAFF02C0EEFF03C0EDFFF36A030E68
:1042E000E15EE7CFD9FF1200D9CFE6FFE1CFD9FFDA
:1042F000080EE126010EDB6A030ED926DE6ADD6AAE
:10430000D95EDF6AE66EE66A890E006E730E016E94
:104310000001026B00C0E6FF01C0E6FF02C0E6FF3D
:10432000FD0EDBCF03F0E828DBCF04F003C0E6FF8F
:1043300004C0E6FFF0EC37F0070EE15EF3500DE14C
:10434000D9CFE9FFDACFEAFFFD0EE926040EEE260B
:10435000000EED22020EDB6A31D0040EE66EE66A34
:104360008D0E006E730E016E0001026B00C0E6FF41
:1043700001C0E6FF02C0E6FFFD0EDBCF03F0E82838
:10438000DBCF04F003C0E6FF04C0E6FFF0EC37F03B
:10439000070EE15EF35010E1D9CFE9FFDACFEAFF73
:1043A000FD0EE926050EEE26000EED22010EE76E4B
:1043B000020EE7CFDBFF02D0020EF0D1FD0EDBCF05
:1043C000E9FFE828DBCFEAFFEF50200A06E1FD0E07
:1043D000DB2AF4E1FE0EDB2AF1D7FD0EDBCFE9FF8D
:1043E000E828DBCFEAFFEECF00F0050E00C0DBFFD0
:1043F000DB50200A01E10BD1050EDB50E85001E152
:1044000006D1050EDB500D0A01E101D1050EDB508E
:104410000A0A01E1FCD0DFCF00F0F90EDBCFE9FFA3
:10442000E828DBCFEAFFEF50005C01E3F0D0010E9B
:10443000DB50020A60E0030A39E0010A01E0E0D043
:10444000FB0EDBCF02F0E828DBCF03F0DF50020DDC
:10445000F3CF04F0F4CF05F004500224006E0550B1
:104460000320016EFD0EDBCF06F0E828DBCF07F05E
:1044700000C0E9FF01C0EAFF06C0EEFF07C0EDFF84
:10448000FD0EDBCFE9FFE828DBCFEAFFEECF00F03F
:10449000050E00C0DBFFDB502F0AD87404E1050EC7
:1044A000DB505C0AD87401E1ABD040D0FB0EDBCF0F
:1044B00002F0E828DBCF03F0DF50DF2A020DF3CF54
:1044C00004F0F4CF05F004500224006E05500320E0
:1044D000016EFD0EDBCF06F0E828DBCF07F000C051
:1044E000E9FF01C0EAFF06C0EEFF07C0EDFF020EC4
:1044F000E76E010E1DD0FD0EDBCFE9FFE828DBCF14
:10450000EAFFEECF00F0050E00C0DBFFDB503F0AF4
:10451000D87404E1050EDB50260AD8740CE0FD0EB9
:10452000DBCFE9FFE828DBCFEAFFEF6A010EE76E99
:10453000E7CFDBFF65D0050EDB502B0A09E1FD0E4E
:10454000DBCFE9FFE828DBCFEAFF200EEF6E58D083
:10455000050EDB502E0A01E014D0DF50010A01E005
:1045600010D0FD0EDB2ADBCF00F0FE0E01E1DB2ACE
:10457000DBCF01F0030E00C0DBFF040E01C0DBFF48
:104580003FD0050EDB503D0A0CE1FD0EDBCFE9FF0D
:10459000E828DBCFEAFFEF6A010EE76EE7CFDBFF2B
:1045A0002FD0050EDB502F0AD87404E1050EDB5026
:1045B0005C0AD87425E0FB0EDBCF02F0E828DBCFE5
:1045C00003F0DF50FF0F020DF3CF04F0F4CF05F03E
:1045D00004500224006E05500320016EFD0EDBCF57
:1045E00006F0E828DBCF07F0010E0626000E0722B2
:1045F00000C0E9FF01C0EAFF06C0EEFF07C0EDFF03
:10460000FD0EDB2A01E0E9D6FE0EDB2AE6D6FD0E22
:10461000DBCFE9FFE828DBCFEAFFEF6AF70EDBCF5D
:10462000E9FFE828DBCFEAFF070EEF6ED9CFE9FFFD
:10463000DACFEAFF030EE926EE5001E1ED5064E027
:10464000030EDBCF02F0E828DBCF03F002C0E6FF69
:1046500003C0E6FF96EC38F0F4CF01F0F3CF00F0A2
:10466000E550E550030E00C0DBFF040E01C0DBFF88
:10467000BC0E006E720E016E060E00C0DBFF070E50
:1046800001C0DBFF050EDB6A050EDB50F90F3CE2D3
:10469000030EE66EE66A060EDBCF00F0E828DBCFFD
:1046A00001F00001026B00C0E6FF01C0E6FF02C09E
:1046B000E6FF030EDBCF03F0E828DBCF04F003C0F6
:1046C000E6FF04C0E6FFF0EC37F0070EE15EF350C2
:1046D0000EE1F70EDBCF00F0E828DBCF01F0050E8E
:1046E000DB5000C0E9FF01C0EAFFEF6E0DD0D9CF6B
:1046F000E9FFDACFEAFF060EE926040EEE26000EE9
:10470000ED22050EDB2AC0D7DF50E86639D0090E4E
:10471000E66EE66A920E006E730E016E0001026B89
:1047200000C0E6FF01C0E6FF02C0E6FFFB0EDBCFE4
:10473000E9FFE828DBCFEAFFEECF03F0EECF04F08D
:1047400003C0E6FF04C0E6FF3BEC38F0070EE15E75
:10475000FB0EDBCFE9FFE828DBCFEAFFEE50EDCF21
:10476000EAFFE96E090EE926000EEA22EF6AF70E6B
:10477000DBCFE9FFE828DBCFEAFF010EEF6EDF2A8F
:10478000F90EDBCF00F0E828DBCF01F0DF5000C0EE
:10479000E9FF01C0EAFFEF6E020EDB50F36E090E77
:0847A000E15EE7CFD9FF120032
:0847A800D9CFE6FFE1CFD9FFF4
:1047B000310EE126140EE66EE66AD9CF00F0DACFAC
:1047C00001F0080E002600C0E6FF01C0E6FF29EC5C
:1047D00028F0040EE15E080EDB50F00B400A01E009
:1047E00042D1080EDB500F0B3F0BE846E846EC0FBA
:1047F000006E1C0E00C0DBFFDB50140801E233D159
:104800001C0EDB50000816E21C0EDBCF00F0016A24
:1048100000C0E6FF01C0E6FFD9CF02F0DACF03F017
:104820001D0E022602C0E6FF03C0E6FF29EC28F0B9
:10483000040EE15E120EDBCF00F0E828DBCF01F0C2
:1048400000C0DFFF010E01C0DBFF120ED926DE6AB9
:10485000DD6AD95E140EE66EE66AD9CF02F0DACFD1
:1048600003F0080E022602C0E6FF03C0E6FF71EC6B
:1048700031F0F4CF01F0F3CF00F0040EE15E001E42
:10488000011E00C0DBFF050E01C0DBFF1C0EDB506C
:10489000000823E21C0EDBCF02F0036A02C0E6FF31
:1048A00003C0E6FFD9CF04F0DACF05F01D0E0426D1
:1048B00004C0E6FF05C0E6FF71EC31F0F4CF01F073
:1048C000F3CF00F0040EE15E001E011E060E00C0D4
:1048D000DBFF070E01C0DBFF05D0060ED926DE6A1E
:1048E000DD6AD95E040EE66EE66AD9CF02F0DACF51
:1048F00003F0022602C0E6FF03C0E6FF71EC31F0D0
:10490000F4CF01F0F3CF00F0040EE15E020E00C020
:10491000DBFF030E01C0DBFFD9CF00F0DACF01F0DF
:10492000080E002600C0E6FF01C0E6FFF9EC25F006
:10493000E550E550000EDBCF00F0E828DBCF01F0BA
:10494000020EDBCF02F0E828DBCF03F00050025C60
:1049500007E10150035804E1080EDB50F00B400A58
:1049600001E081D0D9CFE9FFDACFEAFFFD0EE926D9
:10497000EE5001E1ED5022E0FD0EDBCFE9FFE8282B
:10498000DBCFEAFFE9CF00F0EACF01F0180EDBCF72
:1049900002F0190EDBCF03F01A0EDBCF04F01B0E72
:1049A000DBCF05F000C0E9FF01C0EAFF02C0EEFF67
:1049B00003C0EEFF04C0EEFF05C0EFFFFB0EDBCF30
:1049C000E9FFE828DBCFEAFF060EE926000EEA221F
:1049D000E9CF00F0EACF01F0140EDBCF02F0150EA4
:1049E000DBCF03F0160EDBCF04F0170EDBCF05F0A4
:1049F00000C0E9FF01C0EAFF02C0EEFF03C0EEFF06
:104A000004C0EEFF05C0EFFFF90EDBCF00F0E82891
:104A1000DBCF01F0110EDB5000C0E9FF01C0EAFF5F
:104A2000EF6EF70EDBCF00F0E828DBCF01F00A0EC7
:104A3000DBCF04F0E828DBCF05F01C0EDB50045C74
:104A4000026E0550036A0356140E025E000E035AEE
:104A500000C0E9FF01C0EAFF02C0EEFF03C0EDFFA6
:104A6000010EF36E03D05FEC28F0F36A320EE15EC4
:104A7000E7CFD9FF1200D9CFE6FFE1CFD9FF140E5F
:104A8000E126450EDF6E010EDB6AFA0EDBCF00F089
:104A9000E828DBCF01F0140E0026000E0122020EE2
:104AA00000C0DBFF030E01C0DBFF0101FE4BFF2B4B
:104AB000040EFEC1DBFF050EFFC1DBFF060ED9268B
:104AC000DE6ADD6AD95E640EE76E080EE7CFDBFFB3
:104AD000FC0EDBCF00F0090E00C0DBFF0A0ED9266A
:104AE000DE6ADD6AD95E0C0E00C2DBFF0D0E01C26C
:104AF000DBFF0E0E02C2DBFF0F0E03C2DBFFFD0E5B
:104B0000DBCFE9FFE828DBCFEAFF060EE926000E3F
:104B1000EA22EECF00F0EECF01F0EECF02F0EECFC2
:104B200003F0100E00C0DBFF110E01C0DBFF120E00
:104B300002C0DBFF130E03C0DBFFD9CF00F0DACFDA
:104B400001F000C0E6FF01C0E6FFF9EC25F0E550FA
:104B5000E550140EE66EE66AD9CF02F0DACF03F024
:104B600002C0E6FF03C0E6FF71EC31F0F4CF01F0C4
:104B7000F3CF00F0040EE15E0A0E00C0DBFF0B0E67
:104B800001C0DBFFFA0EDBCF00F0E828DBCF01F03D
:104B9000140E0026000E012200C0E6FF01C0E6FF51
:104BA000E66AFD0EDBCFE9FFE828DBCFEAFFE9CFBD
:104BB00002F0EACF03F002C0E6FF03C0E6FF72ECAA
:104BC00028F0050EE15E140EE66EE66AD9CF00F01D
:104BD000DACF01F000C0E6FF01C0E6FFBCEC28F030
:104BE000040EE15EF36AF46A150EE15EE7CFD9FFC9
:104BF0001200D9CFE6FFE1CFD9FFFD0EDBCFE9FFF1
:104C0000E828DBCFEAFFEE52EE52E9CF00F0EACF20
:104C100001F000C0E6FF01C0E6FFFD0EDBCFE9FFBB
:104C2000E828DBCFEAFFEE52EE52EECF04F0EECFF3
:104C300005F004C0E6FF05C0E6FF8BEC30F0F4CFD2
:104C400003F0F3CF02F0E550E550E550E5CF01F079
:104C5000E7CF00F000C0E9FF01C0EAFF02C0EEFFAD
:104C600003C0EDFFFD0EDBCFE9FFE828DBCFEAFF55
:104C7000040EE926000EEA22E9CF00F0EACF01F0A7
:104C800000C0E6FF01C0E6FFFD0EDBCFE9FFE8282C
:104C9000DBCFEAFF040EE926000EEA22EECF04F095
:104CA000EECF05F004C0E6FF05C0E6FF8BEC30F068
:104CB000F4CF03F0F3CF02F0E550E550E550E5CF37
:104CC00001F0E7CF00F000C0E9FF01C0EAFF02C039
:104CD000EEFF03C0EDFFFD0EDBCFE9FFE828DBCFE1
:104CE000EAFF0A0EE926000EEA22E9CF00F0EACF39
:104CF00001F000C0E6FF01C0E6FFFD0EDBCFE9FFDB
:104D0000E828DBCFEAFF0A0EE926000EEA22EECF02
:104D100004F0EECF05F004C0E6FF05C0E6FF8BEC23
:104D200030F0F4CF03F0F3CF02F0E550E550E5505A
:104D3000E5CF01F0E7CF00F000C0E9FF01C0EAFFD6
:104D400002C0EEFF03C0EDFFE552E7CFD9FF12002E
:104D50009EAA8FD09DAA8DD0AB50060B05E0AB98D4
:104D6000AB880201050E346FAECF32F202013691EC
:104D70003451050A47E0010A35E0070A22E0010A3A
:104D800018E0030A10E002C333F2356BC00E326341
:104D900003D0030E346F39D0410E326336D03681E2
:104DA000020E346F32D036810D0E32632ED0368330
:104DB0002CD03681540E326302D0010E08D0050E7D
:104DC00006D03681DB0E326304D03691040E346F88
:104DD0001CD0C00E326319D0355102E0368315D095
:104DE000369113D03681030E346FDC0E326302D05D
:104DF000C00E04D0DD0E326303D0DB0E326F05D05F
:104E0000369102D033C202F3346B36A11ED00301B7
:104E1000022BFA0E025D01E3026B0251005D10E00D
:104E20000201352B040E006E030E016E03010251C8
:104E3000EA6A0024E96E0150EA2232C2EFFF05D08F
:104E400033C202F30201346B3693020136A311D050
:104E50003693040E006E030E016E3351EA6A00248D
:104E6000E96E0150EA2202C3EFFF0301012B0201A8
:104E7000346B9EA845D09DA843D00401005139E071
:104E8000040E006E040E016E0151EA6A0024E96E00
:104E90000150EA22EECF32F2C00E0201326310D08E
:104EA000DB0E326F040E006E040E016E0401015120
:104EB000EA6A0024E96E0150EA22DC0EEF6E16D099
:104EC000DB0E326310D0DB0E326F040E006E040E68
:104ED000016E04010151EA6A0024E96E0150EA22E0
:104EE000DD0EEF6E03D004010007012B32C2ADFFCF
:104EF00007D09D9803A102D0039102D0C00EAD6EE1
:104F00001200E66AE9EC28F0E5500201346B366BDA
:104F10000301006B016B036B026B0201316B9E9A04
:104F20009D8A9D98200EAC6E900EAB6E070EAF6EF4
:104F3000F28EF28C1200FA0E0401005D01E304D03F
:104F40009DB802D0010E01D0000EF36E1200D9CF31
:104F5000E6FFE1CFD9FF0201010E316F03010151DC
:104F60003EE000C303F3032BFA0E035D01E3036B82
:104F7000040E006E030E016E0351EA6A0024E96E0E
:104F80000150EA22EF50410A20E15FEC28F00401D1
:104F90000381040E006F026B0201316B4F0EE66E4F
:104FA00086EC28F0E5504B0EE66E86EC28F0E550D6
:104FB0000D0EE66E86EC28F0E5500A0EE66E86ECE5
:104FC00028F0E550E0EC28F00AD0FB0EDBCFE9FF3B
:104FD000E828DBCFEAFFEF6A010EF36E01D0F36A37
:104FE000E552E7CFD9FF1200D9CFE6FFE1CFD9FFD5
:104FF000010EE1260201315115E0040E016E030E8F
:10500000026E03010351032BEA6A0124E96E025088
:10501000EA22EECF00F000C0DFFFFA0E035D12E3DC
:10502000036B10D0040E016E040E026E04010251D7
:10503000022BEA6A0124E96E0250EA22EECF00F068
:1050400000C0DFFFDF50F36E020EE15EE7CFD9FF55
:105050001200D9CFE6FFE1CFD9FFFB0EDBCF00F086
:10506000DB06FC0EDBCF01F001E2DB06005001E1C4
:1050700001501BE0FD0EDBCF00F0DB2AFE0EDBCF84
:1050800001F001E1DB2A00C0E6FF01C0E6FFF4EC1D
:1050900027F0E550E5CF01F0E7CF00F0F35000C076
:1050A000E9FF01C0EAFFEF6ED8D7FB0EDBCFF3FFBD
:1050B000E828DBCFF4FFE552E7CFD9FF12009D9A35
:1050C000030101510DE0040E006E030E016E00514C
:1050D000EA6A0024E96E0150EA22EECF00F30107EC
:1050E0009D8A1200D9CFE6FFE1CFD9FFD9CFE9FFE2
:1050F000DACFEAFFFA0EE926EECF00F40401026BE4
:105100000201316BE552E7CFD9FF1200D9CFE6FF9C
:10511000E1CFD9FF0201315118E0040E026E030EF7
:10512000036E03010351032B016A0224006E035036
:105130000122FE0EDB5000C0E9FF01C0EAFFEF6E66
:10514000FA0E035D15E3036B13D0040E026E040E1A
:10515000036E04010251022B016A0224006E035007
:105160000122FE0EDB5000C0E9FF01C0EAFFEF6E36
:10517000E552E7CFD9FF1200D9CFE6FFE1CFD9FF43
:10518000FB0EDBCF00F0DB06FC0EDBCF01F001E213
:10519000DB06005001E101500FE0FD0EDBCFE9FF1F
:1051A000DB2AFE0EDBCFEAFF01E1DB2AEF50E66EE1
:1051B00086EC28F0E550E4D7E552E7CFD9FF12009E
:1051C0000401026B016B03B102D0C00EAD6E9D886D
:1051D0001200D9CFE6FFE1CFD9FF9DB805D0040179
:1051E000006B026B016B036BE552E7CFD9FF120036
:1051F000D9CFE6FFE1CFD9FFD9CF00F0DACF01F068
:10520000FD0E002600C302F0036A00C0E9FF01C0E2
:10521000EAFF0250EE260350ED22FD0EDB2A02E1EA
:10522000FE0EDB2AFD0EDBCF00F0E828DBCF01F01D
:10523000F90E005C000E01580DE3FD0EDBCF00F00F
:10524000E828DBCF01F0FA0E005E000E015A00C024
:1052500003F308D0D9CFE9FFDACFEAFFFD0EE92644
:10526000EECF03F30201010E316FE552E7CFD9FF14
:105270001200D9CFE6FFE1CFD9FFD9CFE9FFDACFCE
:10528000EAFFFC0EE926EECF02F40201316BE55293
:10529000E7CFD9FF1200D9CFE6FFE1CFD9FFE55222
:1052A000E7CFD9FF1200D9CFE6FFE1CFD9FF010E3A
:1052B000E1269D9A02C3DFFF9D8A030101510DE0A3
:1052C000DFCF00F00051D880005404E2DF50FA082C
:1052D000002504D0DF50005D01D0F80EF36EF46AB3
:0A52E000020EE15EE7CFD9FF1200D5
:0652EA00D9CFE6FFE1CF81
:1052F000D9FF1C0EE126E66EE66AD9CF00F0DACFC0
:1053000001F000C0E6FF01C0E6FF29EC28F0040E22
:10531000E15E5FEC28F0D9CF00F0DACF01F000C0F9
:10532000E6FF01C0E6FF8EEC2BF0E550E550000EE5
:10533000DBCF00F0E828DBCF01F0010E005C13E1C9
:10534000015811E1040EDBCF02F0036A060E025C85
:105350000AE1035808E1050EDBCF04F0056A040EEC
:10536000045C01E1055801E09AD0060EDBCF00F0A5
:10537000E828DBCF01F0020E005C0AE1015808E1E9
:10538000FB0EDBCFE9FFE828DBCFEAFFEF6A1DD099
:10539000060EDBCF00F0E828DBCF01F0010E005C49
:1053A0000BE1015809E1FB0EDBCFE9FFE828DBCF79
:1053B000EAFF010EEF6E09D0FB0EDBCFE9FFE82814
:1053C000DBCFEAFF020EEF6E6AD0180EDB5002014F
:1053D000005D01E064D0190EDB50015D01E05FD09B
:1053E0001A0EDB50025D01E05AD01B0EDB50035D4C
:1053F00001E055D0FD0EDBCFE9FFE828DBCFEAFF67
:10540000E9CF00F0EACF01F0080EDBCF02F0090E81
:10541000DBCF03F00A0EDBCF04F00B0EDBCF05F081
:105420000C0EDBCF06F00D0EDBCF07F000C0E9FF5E
:1054300001C0EAFF02C0EEFF03C0EEFF04C0EEFFB2
:1054400005C0EEFF06C0EEFF07C0EFFFFD0EDBCF8D
:10545000E9FFE828DBCFEAFF060EE926000EEA2284
:10546000E9CF00F0EACF01F00E0EDBCF02F00F0E15
:10547000DBCF03F0100EDBCF04F0110EDBCF05F015
:1054800000C0E9FF01C0EAFF02C0EEFF03C0EEFF6B
:1054900004C0EEFF05C0EFFF010EF36E01D0F36A0A
:1054A0001D0EE15EE7CFD9FF1200D9CFE6FFE1CFB5
:1054B000D9FF1C0EE126010EDE6EDD6A020ED92632
:1054C000DE6A080EDD6E020ED95E060EE76E040E71
:1054D000E7CFDBFFE76E050EE7CFDBFFFC0EDB500F
:1054E000010A14E1060ED926010EDE6EDD6A060EF3
:1054F000D95E120EDB68130EDB68140EDB68150E26
:10550000DB68160EDB68170EDB6833D0060ED92673
:10551000020EDE6EDD6A060ED95EFD0EDBCFE9FF00
:10552000E828DBCFEAFFEECF00F0EECF01F0EECFC0
:1055300002F0EECF03F0EECF04F0EECF05F0EECFA9
:1055400006F0EECF07F0EECF08F0EECF09F0120E26
:1055500000C0DBFF130E01C0DBFF140E02C0DBFF37
:10556000150E03C0DBFF160E04C0DBFF170E05C0CF
:10557000DBFF080E04C2DBFF090E05C2DBFF0A0ECB
:1055800006C2DBFF0B0E07C2DBFF0C0E08C2DBFFFF
:105590000D0E09C2DBFF0E0E00C2DBFF0F0E01C2B3
:1055A000DBFF100E02C2DBFF110E03C2DBFF0E0E8B
:1055B000DBCF01F0FD0EDBCFE9FFE828DBCFEAFF10
:1055C000060EE926000EEA22EF500118006E0201D5
:1055D0000A510014E85041E10F0EDBCF03F0FD0E3D
:1055E000DBCFE9FFE828DBCFEAFF060EE926000E55
:1055F000EA22EE52EF500318026E0B510214E850EB
:105600002CE1100EDBCF05F0FD0EDBCFE9FFE82823
:10561000DBCFEAFF060EE926000EEA22EE52EE523A
:10562000EF500518046E0C510414E85016E1110EE9
:10563000DBCF07F0FD0EDBCFE9FFE828DBCFEAFF89
:10564000060EE926000EEA22EE52EE52EE52EF501E
:105650000718066E0D510614E8500DE0180E0EC224
:10566000DBFF190E0FC2DBFF1A0E10C2DBFF1B0E91
:1056700011C2DBFF1ED0FD0EDBCFE9FFE828DBCF38
:10568000EAFF060EE926000EEA22EECF00F0EECF8A
:1056900001F0EECF02F0EECF03F0180E00C0DBFFFA
:1056A000190E01C0DBFF1A0E02C0DBFF1B0E03C088
:1056B000DBFFD9CF00F0DACF01F000C0E6FF01C078
:1056C000E6FF8EEC2BF0E550E5501C0EE66EE66A28
:1056D000060EE66ED9CF00F0DACF01F0120E0026EA
:1056E00000C0E6FF01C0E6FF72EC28F0050EE15EA7
:1056F0001C0EE66EE66AD9CF00F0DACF01F000C0EA
:10570000E6FF01C0E6FFBCEC28F0040EE15EE0EC31
:1057100028F01D0EE15EE7CFD9FF1200D9CFE6FFDA
:10572000E1CFD9FFFD0EDBCFE9FFE828DBCFEAFFB1
:10573000E9CF00F0EACF01F000C0E6FF01C0E6FFCC
:10574000FD0EDBCFE9FFE828DBCFEAFFEECF04F068
:10575000EECF05F004C0E6FF05C0E6FF8BEC30F0AD
:10576000F4CF03F0F3CF02F0E550E550E550E5CF7C
:1057700001F0E7CF00F000C0E9FF01C0EAFF02C07E
:10578000EEFF03C0EDFFFD0EDBCFE9FFE828DBCF26
:10579000EAFFEE52EE52E9CF00F0EACF01F000C08E
:1057A000E6FF01C0E6FFFD0EDBCFE9FFE828DBCF17
:1057B000EAFFEE52EE52EECF04F0EECF05F004C059
:1057C000E6FF05C0E6FF8BEC30F0F4CF03F0F3CF3B
:1057D00002F0E550E550E550E5CF01F0E7CF00F0ED
:1057E00000C0E9FF01C0EAFF02C0EEFF03C0EDFF09
:1057F000FD0EDBCFE9FFE828DBCFEAFF060EE92646
:10580000000EEA22E9CF00F0EACF01F000C0E6FF87
:1058100001C0E6FFFD0EDBCFE9FFE828DBCFEAFFA2
:10582000060EE926000EEA22EECF04F0EECF05F0D8
:1058300004C0E6FF05C0E6FF8BEC30F0F4CF03F0C8
:10584000F3CF02F0E550E550E550E5CF01F0E7CFAA
:1058500000F000C0E9FF01C0EAFF02C0EEFF03C094
:0A586000EDFFE552E7CFD9FF12007B
:06586A00D9CFE6FFE1CFFB
:10587000D9FF300EE126080EE66EE66AD9CF00F0B9
:10588000DACF01F000C0E6FF01C0E6FF29EC28F006
:10589000040EE15E020EDBCF00F0E828DBCF01F062
:1058A0002E0E00C0DBFF2F0E01C0DBFF020ED9263B
:1058B000DE6ADD6AD95E080EE66EE66AD9CF02F0CE
:1058C000DACF03F002C0E6FF03C0E6FF71EC31F06F
:1058D000F4CF01F0F3CF00F0040EE15E001E011ED4
:1058E000280E00C0DBFF290E01C0DBFFF90EDBCF65
:1058F000E9FFE828DBCFEAFF080EEF5EF90EDBCF09
:10590000E9FFE828DBCFEAFFEECF00F0016A00C034
:10591000E6FF01C0E6FFFB0EDBCF02F0E828DBCF9D
:1059200003F002C0E6FF03C0E6FF29EC28F0040EF6
:10593000E15EF90EDBCFE9FFE828DBCFEAFFEECF2F
:1059400002F0036A02C0E6FF03C0E6FFFB0EDBCFF6
:1059500004F0E828DBCF05F004C0E6FF05C0E6FF51
:1059600071EC31F0F4CF01F0F3CF00F0040EE15E02
:10597000001E011E2A0E00C0DBFF2B0E01C0DBFF44
:10598000040EE66EE66AD9CF02F0DACF03F0280EF5
:10599000022602C0E6FF03C0E6FF71EC31F0F4CF4F
:1059A00001F0F3CF00F0040EE15E2C0E00C0DBFF2F
:1059B0002D0E01C0DBFFD9CF00F0DACF01F000C01F
:1059C000E6FF01C0E6FFEAEC2DF0E550E550FD0EE4
:1059D000DBCF00F0E828DBCF01F0DF5000C0E9FFAB
:1059E00001C0EAFFEF6EF70EDBCF00F0E828DBCF57
:1059F00001F0040EDBCF02F0E828DBCF03F000C09B
:105A0000E9FF01C0EAFF02C0EEFF03C0EDFFF50EA3
:105A1000DBCF00F0E828DBCF01F0060EDBCF02F091
:105A2000E828DBCF03F000C0E9FF01C0EAFF02C0B5
:105A3000EEFF03C0EDFF2C0EDBCF00F0E828DBCF3C
:105A400001F02E0EDBCF02F0E828DBCF03F0005090
:105A5000025C04E10150035801E102D0000E01D0C4
:105A6000010EF36E310EE15EE7CFD9FF1200D9CF00
:105A7000E6FFE1CFD9FF280EE126010EDB6AFC0E1E
:105A8000DBCF00F000C0DFFF020ED926DE6ADD6A40
:105A9000D95EF70EDBCF00F0E828DBCF01F0040E73
:105AA00000C0DBFF050E01C0DBFFF50EDBCF00F011
:105AB000E828DBCF01F0060E00C0DBFF070E01C0B7
:105AC000DBFFF90EDBCF00F0016A00C0E6FF01C08A
:105AD000E6FFFA0EDBCF02F0E828DBCF03F002C0CE
:105AE000E6FF03C0E6FFD9CF04F0DACF05F0080ED9
:105AF000042604C0E6FF05C0E6FF10EC38F0060EF1
:105B0000E15ED9CF00F0DACF01F000C0E6FF01C0BE
:105B1000E6FFEAEC2DF0E550E550F90EDBCF02F0A0
:105B2000036A080E0226000E032202C0E6FF03C02D
:105B3000E6FFD9CF04F0DACF05F004C0E6FF05C0D8
:105B4000E6FF71EC31F0F4CF01F0F3CF00F0040E7A
:105B5000E15E020E00C0DBFF030E01C0DBFFF90EA9
:105B6000DBCF00F0016A080E0026000E012200C003
:105B7000E6FF01C0E6FF010EE66EFD0EDBCF02F090
:105B8000E828DBCF03F002C0E6FF03C0E6FF3BECF2
:105B900025F0050EE15EF90EDBCF00F0016A080E7C
:105BA0000026000E012200C0E6FF01C0E6FFD9CFAB
:105BB00002F0DACF03F002C0E6FF03C0E6FFBCEC60
:105BC00028F0040EE15EE0EC28F0290EE15EE7CF5C
:105BD000D9FF1200D9CFE6FFE1CFD9FFFD0EDBCF11
:105BE000E9FFE828DBCFEAFF040EE926000EEA22EF
:105BF000E9CF00F0EACF01F000C0E6FF01C0E6FF08
:105C0000FD0EDBCFE9FFE828DBCFEAFF040EE92633
:105C1000000EEA22EECF04F0EECF05F004C0E6FF5E
:105C200005C0E6FF8BEC30F0F4CF03F0F3CF02F0C9
:105C3000E550E550E550E5CF01F0E7CF00F000C0BA
:105C4000E9FF01C0EAFF02C0EEFF03C0EDFFFD0E59
:105C5000DBCFE9FFE828DBCFEAFF060EE926000EDE
:105C6000EA22E9CF00F0EACF01F000C0E6FF01C070
:105C7000E6FFFD0EDBCFE9FFE828DBCFEAFF060EEB
:105C8000E926000EEA22EECF04F0EECF05F004C0C4
:105C9000E6FF05C0E6FF8BEC30F0F4CF03F0F3CF66
:105CA00002F0E550E550E550E5CF01F0E7CF00F018
:105CB00000C0E9FF01C0EAFF02C0EEFF03C0EDFF34
:105CC000FD0EDBCFE9FFE828DBCFEAFFEE52EE5214
:105CD000E9CF00F0EACF01F000C0E6FF01C0E6FF27
:105CE000FD0EDBCFE9FFE828DBCFEAFFEE52EE52F4
:105CF000EECF04F0EECF05F004C0E6FF05C0E6FFEE
:105D00008BEC30F0F4CF03F0F3CF02F0E550E55028
:105D1000E550E5CF01F0E7CF00F000C0E9FF01C09A
:105D2000EAFF02C0EEFF03C0EDFFE552E7CFD9FF67
:025D300012005F
:0E5D3200D9CFE6FFE1CFD9FF3F0EC716C66AF4
:105D4000C56AC686000EC71294869488C68AFE0E5F
:105D5000DB50C86EE552E7CFD9FF1200D9CFE6FF7E
:105D6000E1CFD9FF020EE126FC0EDBCF00F0E828E0
:105D7000DBCF01F000C0DFFF010E01C0DBFFC5502B
:105D80001F0B006E000EC7B4010E0010E85001E0BA
:105D9000F6D7C580C5A001D0FDD7A1A601D02FD0D0
:105DA000FE0EDB50E66E71EC30F0E550F35001E092
:105DB00026D0C5501F0B006E000EC7B4010E001098
:105DC000E85001E0F6D7C5BC2AD0010EDB50E66EE4
:105DD00071EC30F0E550F35001E011D0C5501F0BCD
:105DE000006E000EC7B4010E0010E85001E0F6D7B7
:105DF000DF50E66E71EC30F0E550F35002E0010E3A
:105E00000FD0C5501F0B006E000EC7B4010E00105E
:105E1000E85001E0F6D7C5BC02D0F36A02D0020E0A
:105E2000F36E030EE15EE7CFD9FF1200D9CFE6FF94
:105E3000E1CFD9FF010EE126FC0EDBCF01F0E8280F
:105E4000DBCF02F001C0E6FF02C0E6FFFE0EDB5032
:105E5000E66EAEEC2EF0E550E550E550F3CF00F0E5
:105E600000C0DFFFDF50E85001E009D01AEC30F04D
:105E7000F3CF00F000C0DFFFDF50E85002E0DF505A
:105E80002BD0C5501F0B006E000EC7B4010E0010C2
:105E9000E85001E0F6D7C580C5A001D0FDD7A1A686
:105EA00001D009D0FE0EDB50010FE66E71EC30F030
:105EB000E550F35002E0010E0FD0C5501F0B006EED
:105EC000000EC7B4010E0010E85001E0F6D7C5BCC3
:105ED00002D0F36A02D0020EF36E020EE15EE7CF4B
:105EE000D9FF1200D9CFE6FFE1CFD9FFC5501F0B74
:105EF000006E000EC7B4010E0010E85001E0F6D7A6
:105F0000FE0EDB50E66E71EC30F0E550F35002E02F
:105F1000010E0FD0C5501F0B006E000EC7B4010E4E
:105F20000010E85001E0F6D7C5BC02D0F36A02D0F9
:105F3000020EF36EE552E7CFD9FF1200C5501F0BDA
:105F4000006E000EC7B4010E0010E85001E0F6D755
:105F5000C584C5A401D0FDD7F36A120084EC30F0EB
:105F6000C5A601D0FDD7C59AC588C5A801D0FDD763
:105F7000C950F36E120084EC30F0C5A601D0FDD7F5
:105F8000C58AC588C5A801D0FDD7C584C5A401D0E0
:105F9000FDD7F36A1200D9CFE6FFE1CFD9FF010E9A
:105FA000E126FC0EDBCF01F0E828DBCF02F001C0D8
:105FB000E6FF02C0E6FFFE0EDB50E66E16EC2FF0A9
:105FC000E550E550E550F3CF00F000C0DFFFDF50B3
:105FD000E85001E028D0F90EDBCFE9FFDB06E950FD
:105FE000E8501BE0FA0EDBCF00F0DB2AFB0EDBCF24
:105FF00001F001E1DB2A00C0E6FF01C0E6FFAEECE4
:106000002FF0E550E5CF01F0E7CF00F0F35000C0EE
:10601000E9FF01C0EAFFEF6EDED7BBEC2FF0F3CF54
:1060200000F000C0DFFFDF50F36E020EE15EE7CF4D
:10603000D9FF1200C5501F0B006E000EC7B4010E31
:106040000010E85001E0F6D7C584C5A401D0FDD703
:10605000A1A603D0010EF36E01D0F36A1200D9CFCE
:10606000E6FFE1CFD9FF010EE126C5501F0B006E00
:10607000000EC7B4010E0010E85001E0F6D7C5804D
:10608000C5A001D0FDD7A1A601D022D0FE0EDB50C5
:10609000E66E71EC30F0E550F35001E019D0C550D8
:1060A0001F0B006E000EC7B4010E0010E85001E097
:1060B000F6D7A1A601D00CD0C5BC02D0DF6A02D0B1
:1060C000040EDF6EC584C5A401D0FDD7A1A602D001
:1060D000010E01D0DF50F36E020EE15EE7CFD9FF73
:1060E0001200D9CFE6FFE1CFD9FFFE0EDB50C96E1B
:1060F000C6AE02D0F36804D0C7A001D0FDD7F36AC2
:10610000E552E7CFD9FF1200C586C7B001D0FDD751
:06611000C950F36E1200FD
:0A611600D9CFE6FFE1CFD9FF030E59
:10612000E126FD0EDBCF00F0E828DBCF01F000C058
:10613000DFFF010E01C0DBFFDBCF00F0020E00C06D
:10614000DBFFDFCF00F0010E00C0DBFF020EDBCF74
:1061500000F000C0DFFF000EDBCFF3FFE828DBCF4D
:10616000F4FF040EE15EE7CFD9FF1200D9CFE6FFBE
:10617000E1CFD9FF070EE126FB0EDBCF00F0FC0ECE
:10618000DBCF01F0FD0EDBCF02F0FE0EDBCF03F024
:10619000010E00C0DBFF020E01C0DBFF030E02C0D8
:1061A000DBFF040E03C0DBFFD9CF00F0DACF01F034
:1061B000010E0026050E00C0DBFF060E01C0DBFF4E
:1061C000050EDBCFE9FFE828DBCFEAFFEE52EE5207
:1061D000EE52EECF00F000C0DFFF050EDBCFE9FF8F
:1061E000E828DBCFEAFFE9CF00F0EACF01F0030EA9
:1061F0000026000E0122050EDBCFE9FFE828DBCFE9
:10620000EAFFEF5000C0E9FF01C0EAFFEF6E050EA4
:10621000DBCFE9FFE828DBCFEAFFE9CF00F0EACFE8
:1062200001F0DF5000C0E9FF01C0EAFFEF6E050E8C
:10623000DBCFE9FFE828DBCFEAFFEE52EE52EECFEC
:1062400000F000C0DFFF050EDBCFE9FFE828DBCF61
:10625000EAFFE9CF00F0EACF01F0020E0026000EBF
:106260000122050EDBCFE9FFE828DBCFEAFFEE5283
:10627000EF5000C0E9FF01C0EAFFEF6E050EDBCF73
:10628000E9FFE828DBCFEAFFE9CF00F0EACF01F031
:10629000010E0026000E0122DF5000C0E9FF01C000
:1062A000EAFFEF6E010EDBCF00F0020EDBCF01F054
:1062B000030EDBCF02F0040EDBCF03F0020ED95C3D
:1062C000E96E000EDA58EA6E03C0EDFF02C0EDFF82
:1062D00001C0EDFF00C0EFFF080EE15EE7CFD9FF80
:1062E0001200D9CFE6FFE1CFD9FF0A0EE126DE6A20
:1062F000DE6ADE6ADD6ADD52DD52FB0EDBCF02F0C4
:10630000E828DBCF03F002C000F003C001F0D89012
:1063100001320032040E00C0DBFF050E01C0DBFFBE
:10632000FD0EDBCF00F0E828DBCF01F0060E00C049
:10633000DBFF070E01C0DBFF040EDBCF00F0DB0646
:10634000050EDBCF01F001E2DB06005001E1015058
:1063500020E0D9CF00F0DACF01F0060ED926DECF4B
:10636000E9FFDDCFEAFF020EDE26000EDD22060E7B
:10637000D95EEECF02F0EECF03F000C0E9FF01C01E
:10638000EAFF0250EE260350EE22000EEE22EE222D
:10639000D3D7FB0EDBCF00F0E828DBCF01F00050B5
:1063A000010B16E0D9CF00F0DACF01F0060EDBCFFB
:1063B000E9FFE828DBCFEAFFEECF02F000C0E9FFFB
:1063C00001C0EAFF0250EE26000EEE22EE22EE227F
:1063D000D9CFE9FFDACFEAFFEC50ECCF02F0ECCFF7
:1063E00003F0046A056A02C000F003C001F0080E61
:1063F00000C0DBFF090E01C0DBFF005001E10150CE
:106400002CE0DECF04F0DDCF05F0020EDBCF06F08E
:10641000030EDBCF07F0066A076A080EDBCF08F031
:10642000E828DBCF09F000010A6B0B6B085004244D
:10643000006E09500520016E0A500620026E0B50B6
:106440000720036E00C0DEFF01C0DDFF020E02C0A8
:10645000DBFF030E03C0DBFFBBD7D9CFE9FFDACFE9
:10646000EAFFEECFF3FFEECFF4FFF31EF41E0B0EA8
:08647000E15EE7CFD9FF120045
:086478000201386B376B0B0EBB
:10648000E66E99EC2EF0E550010EF36E1200D9CFB6
:10649000E6FFE1CFD9FF120EE126020137A103D0BA
:1064A000F36AF46AB2D00F0ED926200EDE6EDD6AD2
:1064B0000F0ED95EFD0EDBCFE9FFE828DBCFEAFF48
:1064C000EF5001E1A0D0FD0EDBCF02F0E828DBCFDA
:1064D00003F002C0E6FF03C0E6FF96EC38F0F4CF0D
:1064E00001F0F3CF00F0E550E550FD0E00C0DBFFFA
:1064F000FE0E01C0DBFF0F0EE66ED9CF00F0DACF43
:1065000001F000C0E6FF01C0E6FFDBCF02F0E828A3
:10651000DBCF03F002C0E6FF03C0E6FFA00EE66E8D
:10652000CBEC2FF0060EE15EDF50E86652D0FD0E98
:10653000DBCF02F0E828DBCF03F002C0E6FF03C0A8
:10654000E6FF5EEC38F0F4CF01F0F3CF00F0E55059
:10655000E550110E00C0DBFFDB500C0805E20C0E0D
:10656000E76E110EE7CFDBFF110EDBCF00F0016A03
:1065700000C0E6FF01C0E6FFD9CF02F0DACF03F09A
:10658000030E022602C0E6FF03C0E6FFFD0EDBCFCE
:1065900004F0E828DBCF05F004C0E6FF05C0E6FF05
:1065A0006CEC38F0060EE15EF35009E10201382B85
:1065B000010EDBCFF3FFE828DBCFF4FF26D0D9CFE5
:1065C000E9FFDACFEAFF0F0EE926EE26000EED22F4
:1065D00092D7DF50040A17E1010EDBCF00F0E82864
:1065E000DBCF01F0FF0E005C02E1FF0E01580BE073
:1065F000010EDBCF00F0E828DBCF01F00F0E00C06A
:10660000DBFF100E76D7F368F468130EE15EE7CF78
:10661000D9FF120002013B6B3791385101E0380776
:106620001200D9CFE6FFE1CFD9FFFD0EDBCF39F263
:10663000E828DBCF3AF2FD0EDBCF00F0E828DBCF15
:1066400001F000C0E6FF01C0E6FFA00EE66E16EC0A
:106650002FF0E550E550E550F35001E102D0000E77
:1066600001D0010EF36EE552E7CFD9FF1200D9CF6A
:10667000E6FFE1CFD9FF010EE126AEEC2FF0F3CF1C
:1066800000F000C0DFFF0201394B3A2BDF50030A54
:106690000AE1AEEC2FF0F3CF00F000C0DFFF020103
:1066A000394B3A2B05D0DF50040A02E139693A69C7
:1066B000DF50F36E020EE15EE7CFD9FF1200BBECB4
:1066C0002FF039C2F3FF3AC2F4FF12000201378102
:1066D000200EF36EF46A1200D9CFE6FFE1CFD9FFA6
:1066E000FD0EDBCF39F2E828DBCF3AF2D9CFE9FF54
:1066F000DACFEAFFFD0EE926EECF3BF23F0E0201B4
:106700003B17FD0EDBCF00F0E828DBCF01F000C027
:10671000E6FF01C0E6FFA00EE66EAEEC2EF0E550FF
:10672000E550E550F35001E102D0000E01D0010E1A
:10673000F36EE552E7CFD9FF1200D9CFE6FFE1CFE4
:10674000D9FFFE0EDB50E66E72EC2FF0E550F350F1
:1067500002E0F36A16D002013B2B394B3A2B400E74
:106760003B5D0DE3C5EC33F039C2E6FF3AC2E6FF0C
:10677000A00EE66EAEEC2EF0E550E550E550010EB1
:10678000F36EE552E7CFD9FF120002013B6B9EEC9E
:106790002FF0A00EE66E2FEC30F0E550F35001E044
:0C67A000F8D739C2F3FF3AC2F4FF120030
:0467AC00FF0EE3CF2A
:1067B000EAFFE552FF0EE3CFE9FFE552E66AE66A3B
:1067C000D9CFE6FFDACFE6FFFC0EE124D96EFF0E4B
:1067D000E220DA6EE66AE66AE66A200EEF5C06E020
:1067E000090EEF5C03E0EF6603D03FD0EE50F5D723
:1067F0002D0EEF5C03E1FF0EE32A03D02B0EEF5CBE
:1068000001E1EE502F0EEF6424D03A0EEF6021D05C
:10681000D890F90EE336FA0EE336FD0EDECFE3FF35
:10682000FE0EDDCFE3FFD890F90EE336FA0EE33625
:10683000D890F90EE336FA0EE336FD0EE350DE266D
:10684000FE0EE350DD22300EEE5CDE26000EDD2271
:10685000D9D7FF0EE3CFE8FFE85207E0F90EE31EB9
:10686000E32AFA0ED8B4E306E31EE552E552E552F8
:10687000FF0EE3CFDAFFE552FF0EE3CFD9FFE5527B
:10688000E1CFE9FFE2CFEAFFED52ED52EECFF3FFA9
:10689000EFCFF4FF1200D9CFE6FFDACFE6FFFA0E12
:1068A000E3CFD9FFFB0EE3CFDAFFFD0EE35209E79A
:1068B0002D0EDE6EFC0EE31EE32AFD0ED8B4E306B9
:1068C000E31EE652E652E652FD0EE124E76EFF0EAD
:1068D000E220E46EE652F70EE3CFE6FFF70EE3CFD9
:1068E000E6FFBBEC34F0F90EE124E96EFF0EE22086
:1068F000EA6EABEC34F00AE1A8EC34F009E1ABEC61
:1069000034F008E1A8EC34F007E108D0B6EC34F03C
:10691000B1EC34F0B6EC34F0B1EC34F0B6EC34F069
:10692000DE6AF90EE126FF0EE222FF0EE3CFDAFF68
:10693000E552FF0EE3CFD9FFE552FC0EE124E96EEC
:10694000FF0EE220EA6EEECFF3FFEFCFF4FF12006E
:10695000EF380F0B1200EF500F0B02E1EE52D8840C
:106960001200EF380F0B300FDE6E1200EE500F0BDF
:10697000300FDE6E1200FC0EE3CFE9FFFD0EE3CF19
:10698000EAFF100EE66EEE6AEE6AEF6AD890FD0E30
:10699000E336FE0EE336ED36ED36EF36FF0EE30658
:1069A00009E0DCEC34F0EE52DCEC34F0EE52DCECDE
:1069B00034F0EDD7E56E1200030EEF24E8B6EF6E6B
:0A69C000300EEF24E8BEEF6E000C6D
:0669CA000001B26B81EC3C
:1069D00027F01DEC3AF088EC00F01200D9CFE6FF6A
:1069E000E1CFD9FF060EE126010EE76E050EE7CFD7
:1069F000DBFF050EDB5001E1EDD0050EDB6A000187
:106A0000B251040A01E1C7D0070A01E18CD0050A9E
:106A100001E176D0040A3BE0070A32E0050A03E010
:106A2000010A01E0E6D7D9CF00F0DACF01F0040E79
:106A3000002600C0E6FF01C0E6FFB30E026E000EA6
:106A4000036E02C0E6FF03C0E6FFA7EC27F0040ECA
:106A5000E15EF35001E1CDD7010EE76E050EE7CF01
:106A6000DBFF040EDB50E86603D00001020E41D0CC
:106A7000040EDB50060A01E08BD00001050E39D070
:106A8000050EDB6A20EC3AF0F350B3E0A0D0BD0E67
:106A9000E66E000EE66ED9CF00F0DACF01F0040EFC
:106AA000002600C0E6FF01C0E6FFB30EE66E000E52
:106AB000E66ED9CF02F0DACF03F002C0E6FF03C0E2
:106AC000E6FFD4EC23F0080EE15EF35016E0010E71
:106AD000E76E050EE7CFDBFF040EDB50010A03E192
:106AE0000001030E06D0040EDB50060A04E100018B
:106AF000060EB26F7ED7050EDB6A5FEC28F067D01A
:106B0000BDC0E6FFBEC0E6FFB30EE66E000EE66E49
:106B100019EC06F0040EE15EF35002E00001B26BE6
:106B2000050EDB6A66D7B26BBD512908000EBE5553
:106B30002FE3E10EE66E000EE66EDF0EE66E000E4F
:106B4000E66EBD0EE66E000EE66EBF0EE66E000E41
:106B5000E66ED9CF00F0DACF01F0040E002600C0B7
:106B6000E6FF01C0E6FF35EC2CF00A0EE15EF350C3
:106B70000DE0040EDB50080A09E1010EE76E050E78
:106B8000E7CFDBFF0001040EB26F02D00001B26B51
:106B90005FEC28F02ED79BEC27F0F35001E129D7CA
:106BA000E1C0E6FFE2C0E6FFDFC0E6FFE0C0E6FFCF
:106BB000BDC0E6FFBF0EE66E000EE66EE66AB30EDF
:106BC000E66E000EE66E37EC2DF00A0EE15E000177
:106BD000B26B0FD718EC06F0070EE15EE7CFD9FFD6
:026BE0001200A1
:0E6BE200F00E83160F0E9512959A9598929AC2
:106BF000839A8398809A31EC1CF0F00E95168316D8
:106C00008382808A3DEC1CF0809A37EC1CF0F00EF9
:106C100083168382808A3DEC1CF0809A3DEC1CF048
:106C2000F00E83168382808A3DEC1CF0809A0F0E52
:106C30009512280EE66E38EC36F0E550080EE66E3A
:106C400038EC36F0E5500C0EE66E38EC36F0E550D8
:106C5000010EE66E38EC36F0E550130EE66E38ECB9
:106C600036F0E550800EE66E38EC36F0E550120056
:106C7000D9CFE6FFE1CFD9FF65EC36F0F35001E064
:106C8000FBD7959A9598F00E95168316FE0EDB505D
:106C9000F00BE83A8312839A83983DEC1CF0808ACB
:106CA0003DEC1CF0809AF00E8316FE0EDB500F0BAD
:106CB00083123DEC1CF0808A3DEC1CF0809A0F0E94
:106CC0009512E552E7CFD9FF1200959A9598838ADD
:106CD00083983DEC1CF0808A3DEC1CF083A60BD021
:106CE000809A3DEC1CF0808A3DEC1CF0809A839ADF
:106CF000010EF36E09D0809A3DEC1CF0808A3DECC9
:106D00001CF0809A839AF36A1200D9CFE6FFE1CF94
:106D1000D9FF010EE126FD0EDBCFE9FFE828DBCF2E
:106D2000EAFFEECF00F0000E00C0DBFFDB50E850C2
:106D30000BE0DF50E66ECEEC36F0E550FD0EDB2AC0
:106D4000EAE1FE0EDB2AE7D7020EE15EE7CFD9FFCC
:106D50001200D9CFE6FFE1CFD9FF010EE126FD0EEB
:106D6000DBCFF6FFE828DBCFF7FF0A00F5CF00F016
:106D7000000E00C0DBFFDB50E8500BE0DF50E66E9A
:106D8000CEEC36F0E550FD0EDB2AE9E1FE0EDB2A03
:106D9000E6D7020EE15EE7CFD9FF1200D9CFE6FFBA
:106DA000E1CFD9FF65EC36F0F35001E0FBD7959ABF
:106DB0009598F00E95168316FE0EDB50F00BE83A10
:106DC0000F0B83128388839A3DEC1CF0808A3DEC84
:106DD0001CF0809AF00E8316FE0EDB500F0B831210
:106DE0003DEC1CF0808A3DEC1CF0809A0F0E951251
:086DF000E552E7CFD9FF1200C4
:086DF8004D43485053746163E0
:106E00006B2076322E3000426F61726420536574BD
:106E100075702E2E2E0020202020202020202020C3
:106E200020202020202000434F4D4D414E44532E22
:106E300043474900494E4445582E48544D000D0AD9
:106E40000D0A0D4D434850537461636B2044656DCA
:106E50006F204170706C69636174696F6E20763168
:106E60002E3020284D6963726F6368697020544327
:106E7000502F495020537461636B20322E30290DFE
:106E80000A0D0A09313A204368616E676520426F36
:106E90006172642073657269616C206E756D6265E4
:106EA000722E0D0A09323A204368616E67652064CC
:106EB000656661756C742049502061646472657305
:106EC000732E0D0A09333A204368616E67652064AA
:106ED000656661756C74206761746577617920619E
:106EE0006464726573732E0D0A09343A2043686135
:106EF0006E67652064656661756C74207375626E7B
:106F00006574206D61736B2E0D0A09353A20456E4C
:106F100061626C6520444843502026204950204738
:106F20006C65616E696E672E0D0A09363A204469F8
:106F30007361626C652044484350202620495020EC
:106F4000476C65616E696E672E0D0A09373A2044F9
:106F50006F776E6C6F6164204D50465320696D6190
:106F600067652E0D0A09383A205361766520262080
:106F7000517569742E0D0A0D0A456E746572206193
:106F8000206D656E752063686F6963652028312DFB
:106F900038293A20000D0A496E76616C69642069CF
:106FA0006E707574207265636569766564202D2046
:106FB000496E7075742069676E6F7265642E0D0A74
:106FC000507265737320616E79206B657920746FE0
:106FD00020636F6E74696E75652E2E2E0D0A00008B
:106FE000FB0EE3CFF6FFFC0EE3CFF7FFFD0EE3CF82
:106FF000F8FFFE0EE3CFE9FFFF0EE3CFEAFFF90E45
:10700000E35003E1FA0EE35009E0F90EE30602E271
:10701000FA0EE3060900F550EE5CF1E0F36E1200A3
:10702000D9CFE6FFDACFE6FFFA0EE3CFD9FFFB0EAA
:10703000E3CFDAFFFC0EE3CFE9FFFD0EE3CFEAFF7B
:10704000E9CFF3FFEACFF4FFF80EE35003E1F90EC6
:10705000E35008E0F80EE30602E2F90EE306DECFA5
:10706000EEFFF2D7FF0EE3CFDAFFE552FF0EE3CFDC
:10707000D9FFE5521200FB0EE3CFF6FFFC0EE3CF83
:10708000F7FFFD0EE3CFF8FFFE0EE3CFE9FFFF0EA3
:10709000E3CFEAFFE9CFF3FFEACFF4FFF90EE350C5
:1070A00003E1FA0EE35009E0F90EE30602E2FA0EFC
:1070B000E3060900F5CFEEFFF1D71200FE0EE3CF95
:1070C000E9FFFF0EE3CFEAFFF36AF46AEE5203E052
:1070D000F34AF42AFBD71200D9CFE6FFDACFE6FF56
:1070E000FA0EE3CFD9FFFB0EE3CFDAFFFC0EE3CFBE
:1070F000E9FFFD0EE3CFEAFFF80EE35003E1F90EDE
:10710000E3500AE0F80EE30602E2F90EE306DE5071
:10711000EF5C02E1EE66F0D7F36EFF0EE3CFDAFF2D
:10712000E552FF0EE3CFD9FFE5521200FE0EE3CF8A
:10713000E9FFFF0EE3CFEAFFE9CFF3FFEACFF4FF69
:10714000610EEF5C05E67B0EEF5C02E7DF0EEF16EB
:06715000EE52F6E1120010
:0A715600485454502F312E302035DC
:107160003033200D0A0D0A53657276696365205528
:107170006E617661696C61626C650D0A000D0A0DC5
:107180000A00485454502F312E3020323030204FD6
:107190004B0D0A436F6E74656E742D747970653A89
:1071A0002000485454502F312E3020343034204E9B
:1071B0006F7420666F756E640D0A0D0A4E6F742031
:1071C000666F756E642E0D0A000D0A4E6F77207281
:1071D000756E6E696E67206170706C696361746949
:1071E0006F6E2E2E2E000D0A526561647920746F29
:1071F00020646F776E6C6F6164204D504653206938
:107200006D616765202D2055736520586D6F64652D
:107210006D2070726F746F636F6C2E0D0A000D0A13
:1072200044484350202620495020476C65616E69D0
:107230006E672064697361626C65642E0D0A000DCF
:107240000A44484350202620495020476C65616E0F
:10725000696E6720656E61626C65642E0D0A000DB3
:107260000A44656661756C74205375626E6574209E
:107270004D61736B2028000D0A44656661756C745E
:107280002047617465776179204164647265737326
:107290002028000D0A44656661756C7420495020F1
:1072A000416464726573732028000D0A5365726926
:0C72B000616C204E756D62657220280034
:0472BC0054585400CE
:1072C00048544D0047494600434749004A5047004B
:1072D000434C410057415600746578742F706C61BF
:1072E000696E000000000000000000007465787402
:1072F0002F68746D6C0000000000000000000000AA
:10730000696D6167652F6769660000000000000015
:1073100000000000746578742F68746D6C000000C4
:107320000000000000000000696D6167652F6A7051
:107330006567000000000000000000006170706CD4
:1073400069636174696F6E2F6A6176612D766D0075
:10735000617564696F2F782D776176650000000094
:1073600000000000485454502F312E30203230306D
:10737000204F4B0D0A436F6E74656E742D747970D7
:10738000653A20000D0A0D0A0047455400504F533E
:0C7390005400494E4445582E48544D000E
:04739C005A0EF66E21
:1073A000000EF76E000EF86E00010900F550FA6F3E
:1073B0000900F550FB6F03E1FA6701D03DD00900E9
:1073C000F550F56F0900F550F66F0900F550F76FAD
:1073D00009000900F550E96E0900F550EA6E090050
:1073E00009000900F550F86F0900F550F96F090020
:1073F0000900F6CFFCF0F7CFFDF0F8CFFEF0F5C0B6
:10740000F6FFF6C0F7FFF7C0F8FF0001F85302E1FE
:10741000F95307E00900F550EE6EF807F8E2F907B6
:10742000F9D7FCC0F6FFFDC0F7FFFEC0F8FF000172
:0A743000FA07000EFB5BBFD7120045
:06743A000001FF6B1200CF
:10744000D9CFE6FFE1CFD9FF0B0EE1260001FF51B6
:10745000000A01E021D0D9CF00F0DACF01F00A0E06
:10746000002600C0E6FF01C0E6FFD9CF02F0DACF68
:1074700003F002C0E6FF03C0E6FF75EC29F0040E3E
:10748000E15EF35001E11FD00A0EDB50E86601D047
:107490001AD00001010EFF6F9BEC27F0F35011E0B2
:1074A000E66AD9CF00F0DACF01F000C0E6FF01C0F4
:1074B000E6FF55EC2AF0E550E550E5500001FF6B82
:1074C00002D0F36A02D0010EF36E0C0EE15EE7CF3C
:0474D000D9FF1200CE
:0C74D4005E0ED66EF80ED76E070ED56E59
:1074E000D58EF284F28A1200FEC3F3FFFFC3F4FFCD
:1074F0001200F2A40AD0F80ED76E5E0ED66E03010B
:0C750000FE4BFF2B0F018978F294120063
:04750C00FF0EE3503B
:10751000186E480E01D04C0EE76EE72EFED7E76AD4
:0C752000E72EFED7182EF7D7000012004F
:04752C0015EE00F068
:1075300025EE00F0F86A178CCEEC39F0B2EC14F0BE
:04754000FDD7120061
:0C754400FF0EE350E84E1200000000D0E3
:0A75500000D000D0E82EFAD7120098
:06755A000001AA72937209
:0C75600077725F723F721E72E671C97193
:04756C00A271827115
:047570007D71567162
:02757400000015
:02757600000013
:020000040030CA
:08000000FFFAFCFEFFFEFFFF0A
:00000001FF
